:020000040800F2
:102000001033002019210008FF2B000885750008F7
:10201000077A0008FD270008D59D00080000000091
:10202000000000000000000000000000DD8C00083F
:10203000FD2B0008000000008D7B0008BD95000806
:10204000332100083321000833210008377D0008C0
:102050003321000833210008F54D0008D14E000857
:1020600033210008E34E0008F54E00083321000834
:1020700033210008332100083321000833210008F0
:10208000332100083321000833210008E59A0008B5
:10209000AD9B000833210008332100081D4F0008C4
:1020A00033210008332100083321000833210008C0
:1020B0003321000845990008332100083321000826
:1020C00033210008332100083321000833210008A0
:1020D00033210008B59900084D9A00083321000803
:1020E000154E0008332100083321000800000000CD
:1020F00000000000000000000000000000000000E0
:1021000033210008DFF80CD000F07EFB00480047C8
:10211000F1B3000810330020064880470648004706
:10212000FEE7FEE7FEE7FEE7FEE7FEE7FEE7FEE787
:10213000FEE7FEE7E19800080521000840EA0103F8
:102140009B0703D009E008C9121F08C0042AFAD26D
:1021500003E011F8013B00F8013B521EF9D2704731
:10216000D2B201E000F8012B491EFBD270470022D9
:10217000F6E710B513460A4604461946FFF7F0FF86
:10218000204610BD421C10F8011B0029FBD1801A0B
:10219000704730B504460020034600E05B1C9342C4
:1021A00003D2E05CCD5C401BF8D030BD80EA010278
:1021B00010B502F00043400022D04A001FD0010EAB
:1021C00001EB1261C0F35600C2F3560240F4000066
:1021D00042F40002A0FB022000047F39140400D066
:1021E000401C50EA124001D44000491EC2B20C0605
:1021F00004EBD010401C4008802A02D003E00020ED
:1022000010BD20F00100002900DA0020184310BDA5
:102210002DE9FE4F804681EA0300C00F0C46009076
:1022200021F0004123F00045B8EB0200A94105D29E
:102230004046214690461C460B46024623F000408D
:10224000104347D0270DC7F30A00C3F30A51029089
:10225000401A019040286BDAC3F3130040F4801B4E
:102260000098924620B10023D2EB030A63EB0B0BDC
:1022700001985946C0F14002504600F0FAF906466E
:102280000D4650465946019A00F012FA10EB08002C
:102290006141002487EA115284EAE7731A4340D06F
:1022A000009A62B3019A012A4FEA075215DC001B1B
:1022B00061EB02014FF0004202EA0752CDE9004211
:1022C000001C41F5801132462B4600F049FA03B05C
:1022D000BDE8F08F40462146F9E7001B61EB0201A3
:1022E000001C41F5801300185B412018A2F500176F
:1022F00047EB030140EAD570B6196D4111E06D0856
:102300004FEA360645EAC0754FEA0752001B61EBFB
:102310000201001C41F5801149084FEA3000001904
:10232000514132462B4603B0BDE8F04F00F009BAE8
:102330000098012240000023D0EB020263EBE0731F
:10234000009821464FEAE074B8EB000061EB04010D
:10235000E9E783F000435BE781F0004158E72DE9AE
:10236000FE4F81EA030404F0004421F00041009490
:102370004FF0000B23F0004350EA01045ED052EA14
:1023800003045BD0C3F30A54C1F30A552C44A4F2EE
:10239000F3340194A0FB0254C1F3130141F4801102
:1023A000C3F3130343F4801301FB024400FB034E09
:1023B000840A970A44EA815447EA8357A4FB0768D2
:1023C00002958D0A05FB07854FEA932C04FB0C54FC
:1023D0002705029D4FEA065847EA1637B5EB080570
:1023E0006EEB070C870E920E47EA811742EA8312C2
:1023F000A7FB0201B6EB0B0164EB00042B0D43EAD3
:102400000C335E1844EB1C50DA465146E7FB0201E0
:10241000C5F313044FEA0B3343EA14534FEA043273
:10242000019C43EA0603A4F10C040294009CCDE94C
:1024300000B400F095F903B0BDE8F08F002001462C
:10244000F9E72DE9F04D81EA030404F0004B21F097
:10245000004514464FF0000A23F0004150EA0502FF
:1024600020D054EA01021DD0C5F30A570246C5F335
:102470001303C1F31300C1F30A5640F4801543F46B
:102480008013A7EB0608101BD64608F2FD3873EB45
:10249000050002D308F1010801E092185B41B8F190
:1024A000000F03DA00200146BDE8F08D00204FF454
:1024B0008011064684460EE0171B73EB050705D313
:1024C000121B63EB050306434CEA010C49084FEA73
:1024D000300092185B4150EA0107EDD152EA030047
:1024E00012D082EA040083EA0501084305D0101BDC
:1024F000AB4106D20122002306E000224FF0004348
:1025000002E06FF0010253101AEB06004CEB085189
:1025100010EB0A0041EB0B01BDE8F04D00F011B9E2
:10252000C10F80EAE0700844CA079623002100F03A
:10253000DAB80EB540F2334102910021CDE9001125
:102540000A460B4600F00CF903B000BD00F0004253
:1025500020F00040C10DC0F3160040F400007F29B8
:1025600001DA00207047962903DCC1F19601C840CA
:1025700001E096398840002AF4D040427047C1F308
:102580000A5210B5C1F3130140F2FF3341F4801138
:102590009A4201DA002010BD40F233439A42A2F27F
:1025A000334203DC524200F073F810BD904010BD7E
:1025B00030B5041E71F1000404DB4FF000444042CA
:1025C00064EB0101141E73F1000405DB1C464FF09F
:1025D0000043524263EB04038B4208BF824230BD8A
:1025E00030B5041E71F1000404DB4FF0004440429A
:1025F00064EB0101141E73F1000405DB1C464FF06F
:102600000043524263EB0403994208BF904230BD3D
:102610002DE9F05F0546002092469B468846064617
:10262000814640241BE0284641464746224600F0AA
:102630002FF853465A46C01A914110D311461846F6
:10264000224600F016F82D1A67EB01084F46224685
:102650000120002100F00DF817EB00094E41201E6B
:10266000A4F10104DFDC484631462A464346BDE872
:10267000F09F202A04DB203A00FA02F10020704784
:102680009140C2F1200320FA03F3194390407047B0
:10269000202A04DB203A21FA02F00021704721FAB7
:1026A00002F3D040C2F1200291400843194670471E
:1026B000202A06DBCB17203A41FA02F043EAE07306
:1026C00006E041FA02F3D040C2F1200291400843F3
:1026D000194670470029A8BF7047401C490008BF31
:1026E00020F00100704710B4B0FA80FC00FA0CF042
:1026F00050EA010404BF10BC704749B1CCF120047A
:1027000021FA04F411FA0CF118BF01212143084306
:10271000A3EB0C01CB1D4FEA00614FEA102042BF32
:10272000002010BC704700EBC35010440029A4BF28
:1027300010BC7047401C490008BF20F0010010BCCD
:10274000704710B5141E73F1000408DA401C41F103
:10275000000192185B411A4301D120F0010010BD25
:102760002DE9F04D92469B4611B1B1FA81F202E09B
:10277000B0FA80F220329046FFF77BFF04460F4606
:1027800040EA0A0041EA0B0153465A46084313D077
:10279000114653EA010019D0C8F140025046FFF734
:1027A00077FF05460E46504659464246FFF761FF01
:1027B000084305D0012004E020463946BDE8F08DED
:1027C0000020054346EAE0762C4337430A98630528
:1027D000E40AA0EB08000022FD0A44EA47540A304C
:1027E00002D500200146E9E7010510196941DDE93C
:1027F000084500196941BDE8F04DA2E700BFFEE7BA
:102800005053313030000000064C074D06E0E068C0
:1028100040F0010394E8070098471034AC42F6D327
:10282000FFF774FCE4C6000804C7000805480078F8
:1028300000B170470120034908700020488000BFA4
:10284000F7E700004C00002010B510480078D8B120
:102850000E48807800F0010088B94FF480410C48A0
:1028600008F06EFD012804D1002008490870488056
:102870000AE006484088401C0449488004E00348B8
:102880004088401C0149488010BD00004C000020D9
:102890000010014010B504460121204602F0D4F991
:1028A00054B1012009490870002048800022042109
:1028B000074808F09DFC08E0044800210160002260
:1028C0004FF40041034808F093FC10BDD0000020F5
:1028D000000C01400010014010B50D480078A8B967
:1028E0004FF400410B4808F033FD08B9012400E023
:1028F00000244FF48041074808F022FD08B9012068
:1029000000E0002004430CB1002010BD0120FCE7D2
:10291000D00000200010014010B50F480078D0B161
:102920000D484088401C0C4948800846408864286F
:1029300008DB0122D103094808F05AFC06480021AF
:10294000016008E00448807800F001024FF4004183
:10295000024808F04DFC10BDD000002000100140DE
:1029600010B540F2046009F059F94FF440730322A6
:1029700048210F4808F08EFC0821022008F03EFC98
:1029800002220021D00108F05FF94FF4807008F0B6
:10299000BFF90921022008F031FC022200211002B7
:1029A00008F052F94FF4007008F0B2F910BD0000C1
:1029B0000010014010B500F0A9F900F08BFA00F00A
:1029C0003BFAFFF7CDFF10BD28B10121044A117079
:1029D000C821518003E00021014A117051807047E5
:1029E0005400002010B5FFF7E5FF0020FFF7ECFFD3
:1029F00010BD00000020014908707047A8000020A9
:102A0000505331303058585F5630315F3043303298
:102A1000303931350000000000B50521034806F0CB
:102A200047FD024880880249088000BDA0090020B7
:102A30005A00002000B50521034806F039FD024880
:102A400080880249088000BDAA0900205C0000209F
:102A50002DE9F05F4FF0000B36480078012801D0D7
:102A6000BDE8F09F4FF48071334808F069FC0128FD
:102A70001AD132480078012816D1314809F085FB77
:102A8000824640F6C41082450AD94FF0280B002038
:102A90002A49087027490870294809F0EBFB2EE005
:102AA0000220264908702AE04FF48071224808F07D
:102AB00047FC20BB21480078022820D1204809F09B
:102AC00064FB82464FEA5A0A5046FFF732FD8046C1
:102AD0004FF0C0421B4BFFF742FC064600221A4B48
:102AE000FFF7AFFC0446FFF74AFD1FFA80FB00200A
:102AF000124908700F490870114809F0BBFB0F48D4
:102B00000078A8B9114801880088401C0F4A10803D
:102B10000F4820F811B010460088052808DB002077
:102B2000114608800B48006840F48020094908607D
:102B300000BF95E75E000020001001405800002013
:102B4000002C01408FC2D53F0000244050000020DF
:102B5000A00900200000002010B54FF0804009F0CF
:102B600089FB012000F0F2F8074809F088FB0748CC
:102B700009F085FB0021054809F00BFB0120044901
:102B800008700449087010BD00040040002C01408A
:102B9000580000205E00002010B54FF0804009F082
:102BA00069FB022000F0D2F8084809F068FB0848E9
:102BB00009F065FB0021064809F0EBFA0120054900
:102BC000087002200449087010BD00000004004095
:102BD000002C0140580000205E00002010B5024883
:102BE00001F09EF910BD00002806002010B504F089
:102BF000E7FD10BD10B504F04BFE10BD70477047E7
:102C0000417070002DE9F05F4FF0000B36480078FE
:102C1000022801D0BDE8F09F4FF40071334808F05E
:102C20008FFB01281AD132480078012816D131488B
:102C300009F0ABFA824640F6C41082450AD94FF03B
:102C4000280B00202A49087027490870294809F0F4
:102C500011FB2EE00220264908702AE04FF4007193
:102C6000224808F06DFB20BB21480078022820D1C3
:102C7000204809F08AFA82464FEA5A0A5046FFF77E
:102C800058FC80464FF0C0421B4BFFF768FB0646DE
:102C900000221A4BFFF7D5FB0446FFF770FC1FFA22
:102CA00080FB0020124908700F490870114809F094
:102CB000E1FA0F480078A8B9114801880088401C43
:102CC0000F4A10800F4820F811B0104600880528E0
:102CD00008DB0020114608800B48006840F4002003
:102CE0000949086000BF95E75E0000200010014020
:102CF00058000020002C01408FC2D53F0000244026
:102D000052000020AA0900200000002010B540F267
:102D1000036008F083FF00210A4808F021FB4FF40C
:102D2000406303221021084808F0B4FA4FF4806190
:102D3000054808F05BFA4FF40061034808F056FAC2
:102D400010BD000000021800000C014070B588B0F2
:102D50000646012E02D0022E07D102E002246502AF
:102D600005E003244FF4006501E008B070BD00BF2A
:102D700040F2036008F052FF4FF4C06008F04EFFCD
:102D80002B46032218212A4808F084FA01212948F9
:102D900008F0E6FA4FF4E06008F040FF4FF08040A2
:102DA00009F0FAF93520ADF804000020ADF806006E
:102DB000ADF80800312003900020ADF810008DF828
:102DC000120001A94FF0804009F05EFA0020ADF832
:102DD00018000120ADF814000020ADF81A00ADF87D
:102DE0001600ADF81C00ADF81E0005AA21464FF0F4
:102DF000804009F067F8182221464FF0804009F022
:102E000084F9602221464FF0804009F051F90022F8
:102E100021464FF0804009F08BF94FF0804009F0D7
:102E20004BF84FF0804009F02AFA00BF9DE7000000
:102E3000000C0140000218001FB540F20B6008F0C2
:102E4000EDFE104809F0A8F9684609F0A5FA6B20D4
:102E5000ADF800000020ADF80200ADF80400401EFF
:102E600002900020ADF80C008DF80E006946054870
:102E700009F00AFA0121034809F076FA014809F03D
:102E8000F9F91FBD002C014010480078E0B10F484F
:102E90004088401C0D49488008464088C82809DB06
:102EA0000B48006840F48030094908600020074959
:102EB000488009E005484088642805D10448006836
:102EC00040F40030024908607047000054000020C0
:102ED000000000201FB540F2017008F09FFE13486B
:102EE00009F05AF9684609F057FA6B20ADF800006E
:102EF0000020ADF80200ADF804004FF4C870029055
:102F00000020ADF80C008DF80E006946074809F066
:102F1000BBF90121054809F02BFA044809F0AAF988
:102F2000002201211D2008F001FC1FBD000400400B
:102F300010B506480078064908700648002101606F
:102F40000548016004F026FB10BD000010000020C1
:102F50000F000020120000201600002070B5074965
:102F60004868FFF7DDFA05460549FFF71FF90446F3
:102F7000FFF7ECFA01498968081A70BD4007002084
:102F8000CDCCCC3D70B507494868FFF7C9FA054676
:102F90000549FFF70BF90446FFF7D8FA014989689C
:102FA000081A70BDE4080020CDCCCC3D10B5044615
:102FB00004B910BD2078C0F340024FF400510A4814
:102FC00008F016F92078C0F3C0024FF4004106481B
:102FD00008F00EF92078C0F300124FF48041024847
:102FE00008F006F900BFE4E7000C014038B50546DB
:102FF0000024052D77D2DFE805F0EF03EEEDEC00BD
:103000009DF8000020F0010000909DF8000020F0E5
:10301000020000909DF8000020F0040000909DF850
:10302000000020F0080000909DF8000020F0100043
:1030300000906846FFF7BAFF00240DE004F0C6FCDC
:103040004FF6E851884200D809E003F0CDFA0A2093
:1030500007F0E8FD601C84B2B4F5FA7FEEDB00BF38
:10306000B4F5FA7F00DB20E2FE480078052876D22E
:10307000DFE800F0034B4C7C9400FB480078032809
:1030800016D1002402E00A2007F0CCFD2046611C86
:103090008CB20F2803DAF54800780028F3D1F34802
:1030A000007800B1DFE7002004F01CFD48B9DAE742
:1030B000ED480078012803D101F008FA08B1D2E701
:1030C000D1E7002402E00A2007F0ACFD2046611C95
:1030D0008CB20F2803DAE64800780028F3D1E448E0
:1030E000007808B1FEE3B4E3E248007838B9022082
:1030F00004F0A4FC00B9F5E3C82007F093FD01201B
:1031000004F09CFC00B9EDE367E066E0002402E017
:103110000A2007F087FD2046611C8CB20F2803DAD5
:10312000D34800780028F3D1D148007800B1D9E322
:10313000012004F083FC00B9D4E3002402E00A205B
:1031400007F070FD2046611C8CB20F2803DAC748D7
:1031500000780028F3D1C548007808B1C2E337E011
:10316000002004F0BFFC00B9BCE336E0002402E01C
:103170000A2007F057FD2046611C8CB20F2803DAA5
:10318000BA4800780028F3D1B848007800B1A9E324
:10319000002004F0A7FC00B9A4E31EE0B2480078C8
:1031A000032811D1002402E00A2007F03BFD20464D
:1031B000611C8CB20F2803DAAC4800780028F3D1E8
:1031C000002004F08FFC02E0002004F08BFC04E0FF
:1031D00088E3CDE129E120E03CE300BF9DF8000059
:1031E00020F0010000909DF8000020F00200009007
:1031F0009DF8000020F00400001D00909DF80000E4
:1032000020F00800083000909DF8000020F0100029
:1032100000906846FFF7CAFE5BE39DF8000020F0CF
:10322000010000909DF8000020F0020000909DF841
:10323000000020F0040000909DF8000020F008003D
:1032400000909DF8000020F0100000906846FFF705
:10325000ADFE00240DE004F0B9FB4FF6E8518842C2
:1032600000D809E003F0C0F90A2007F0DBFC601C7D
:1032700084B2B4F5FA7FEEDB00BFB4F5FA7F00DB71
:1032800030E378480078052874D2DFE800F0034A7C
:103290007A7B930078480078032816D1002402E056
:1032A0000A2007F0BFFC2046611C8CB20F2803DA0D
:1032B0006F4800780028F3D16D48007800B111E321
:1032C000002004F0BBFB48B90CE36B4800780128F0
:1032D00003D101F0DBF808B104E303E3002402E0CA
:1032E0000A2007F09FFC2046611C8CB20F2803DAED
:1032F0005E4800780028F3D15C48007800B1F1E224
:103300005C48007838B9022004F0ECFB00B9E9E22F
:10331000C82007F087FC012004F0E4FB00B9E1E2DB
:1033200063E0002402E00A2007F07CFC2046611CD8
:103330008CB20F2803DA4D4800780028F3D14B48AF
:10334000007800B1CEE2012004F0CCFB00B9C9E264
:10335000002402E00A2007F065FC2046611C8CB2C4
:103360000F2803DA424800780028F3D1404800785B
:1033700008B1B7E238E0002004F060FB00B9B1E228
:1033800033E032E0002402E00A2007F04BFC204644
:10339000611C8CB20F2803DA354800780028F3D17D
:1033A0003348007800B19DE2002004F047FB00B9EB
:1033B00098E21AE030480078032811D1002402E096
:1033C0000A2007F02FFC2046611C8CB20F2803DA7C
:1033D000274800780028F3D1002004F02FFB02E0FA
:1033E000002004F02BFB00E07CE200BF9DF8000011
:1033F00020F00100401C00909DF8000020F0020029
:10340000801C00909DF8000020F0040000909DF8C2
:10341000000020F0080000909DF8000020F010004F
:1034200000906846FFF7C2FD53E29DF8000020F0CF
:10343000010000909DF8000020F0020000909DF82F
:10344000000020F0040000909DF8000020F008002B
:1034500000909DF8000020F0100000906846FFF7F3
:10346000A5FD0BE0050000203A00002039000020F7
:10347000300000201E0000203100002000240DE05C
:1034800004F0A4FA4FF6E851884200D809E003F0AE
:10349000ABF80A2007F0C6FB601C84B2B4F5FA7FD3
:1034A000EEDB00BFB4F5FA7F00DB1BE2FE480078DC
:1034B00005283AD2DFE800F003041C34350011E29D
:1034C000002402E00A2007F0ADFB2046611C8CB20C
:1034D0000F2803DAF54800780028F3D1F348007884
:1034E00000B1FFE1012004F0FDFA00B9FAE11DE0AE
:1034F000002402E00A2007F095FB2046611C8CB2F4
:103500000F2803DAEA4800780028F3D1E848007869
:1035100000B1E7E1012004F091FA00B9E2E105E031
:1035200004E00A2007F07EFB00E0DBE100BF9DF82D
:10353000000020F00100401C00909DF8000020F0E9
:103540000200801C00909DF8000020F00400001D87
:1035500000909DF8000020F00800083000909DF8D1
:10356000000020F0100000906846FFF71FFDB0E15A
:103570000221002004F00CFB9DF8000020F0010067
:1035800000909DF8000020F0020000909DF80000DF
:1035900020F0040000909DF8000020F0080000904A
:1035A0009DF8000020F0100000906846FFF7FEFC38
:1035B000BD48007805287BD2DFE800F00304468987
:1035C000EF008FE10A2007F02DFB9DF8000020F0AE
:1035D0000100401C00909DF8000020F002000090C7
:1035E0009DF8000020F00400001D00909DF80000F0
:1035F00020F0080000909DF8000020F0100010302E
:1036000000906846FFF7D2FC002402E00A2007F091
:1036100009FB2046611C8CB20F2803DAA34800780E
:103620000028F3D1A148007800B15BE1022004F04A
:1036300059FA00B956E1C82007F0F4FA012004F065
:1036400051FA00B94EE1E0E00A2007F0EBFA9DF8EC
:10365000000020F00100401C00909DF8000020F0C8
:10366000020000909DF8000020F00400001D009072
:103670009DF8000020F0080000909DF8000020F068
:103680001000103000906846FFF790FC002402E024
:103690000A2007F0C7FA2046611C8CB20F2803DA13
:1036A000834800780028F3D18148007808B119E1F7
:1036B000AAE0022004F0C2F900B913E1C82007F023
:1036C000B1FA012004F0BAF900B90BE19DE07948A4
:1036D000806879498968884248D2002402E00A203B
:1036E00007F0A0FA2046611C8CB20F2803DA70485C
:1036F00000780028F3D16E48007800B1F2E0002095
:1037000004F09CF900B9EDE0322007F08BFA0A20B2
:1037100007F088FA9DF8000020F00100401C00909E
:103720009DF8000020F0020000909DF8000020F0BD
:103730000400001D00909DF8000020F0080000909B
:103740009DF8000020F01000103000906846FFF750
:103750002DFC022004F072F900B9C3E0C82007F084
:1037600061FA012004F06AF9F0BBBBE0002402E03A
:103770000A2007F057FA2046611C8CB20F2803DAA2
:103780004A4800780028F3D14848007800B1A9E001
:10379000002004F0A7F908B9A4E034E0322007F0D3
:1037A00041FA0A2007F03EFA9DF8000020F00100DF
:1037B000401C00909DF8000020F0020000909DF851
:1037C000000020F00400001D00909DF8000020F093
:1037D000080000909DF8000020F0100010300090CC
:1037E0006846FFF7E3FB00E00CE0022004F07AF902
:1037F00000B977E0C82007F015FA012004F072F94B
:1038000000B96FE001E000E06CE000BF0A2007F0C3
:1038100009FA9DF8000020F00100401C00909DF87E
:10382000000020F0020000909DF8000020F004004D
:10383000001D00909DF8000020F0080000909DF809
:10384000000020F01000103000906846FFF7AEFB3B
:103850003FE000BF0020FFF71DF89DF8000020F0BA
:10386000010000909DF8000020F0020000909DF8FB
:10387000000020F0040000909DF8000020F00800F7
:1038800000909DF8000020F0100000906846FFF7BF
:103890008DFB002503F08EFFD0B10B20054981F888
:1038A0008C000021034809E00500002039000020B9
:1038B0003000002040070020E4080020C0F89010ED
:1038C0000B201C4981F88C0000211A48C0F8901088
:1038D00000BF00BF18489DF8001001701748057020
:1038E00068B238BD9DF8000020F0010000909DF8FE
:1038F000000020F0020000909DF8000020F004007D
:1039000000909DF8000020F0080000909DF8000055
:1039100020F0100000906846FFF748FB06489DF82D
:10392000001001700020054908700846007840B278
:10393000D7E70000E4080020040000200500002074
:1039400070B5044605251748007808B9002070BDF9
:10395000062C1AD2DFE804F003050A0F141A00201F
:10396000F5E7FFF743F900B1012511E0FFF742F950
:1039700000B102250CE000F0EFFC00B1032507E0E8
:1039800000F018FD00B1042502E000BF0020DEE7D2
:1039900000BF052D01DB0020D9E72846FFF726FBF5
:1039A000C0B2D4E70D0000201848007848B317488B
:1039B0004088401C1549488008464088B0F5967FED
:1039C00009DB0846002101601148006840F480507E
:1039D0000F49086018E00D484088C82806D10C48F7
:1039E000006840F480500A4908600DE007484088AC
:1039F000642809D10648006840F4805004490860F2
:103A000002E0002001494880704700006E0000205D
:103A1000000000201848007848B317484088401C30
:103A20001549488008464088B0F5967F09DB08466E
:103A3000002101601148006840F400500F490860FF
:103A400018E00D484088C82806D10C48006840F4AA
:103A500000500A4908600DE007484088642809D1F1
:103A60000648006840F400500449086002E0002065
:103A700001494880704700008000002000000020BD
:103A800010B55448544909680160544854490968BC
:103A90000160544854490968016054484D494860E0
:103AA00053484E49486053484E49486052480021A7
:103AB0000160416001814FF480715048FEF757FB6F
:103AC0004E484D49486040F2197008F0A7F840F29E
:103AD000036008F0A3F84FF4C06008F09FF84FF4BB
:103AE000807303224821464807F0D4FB4FF400734B
:103AF00003221821424807F0CDFB01214FF4EA10C0
:103B000007F02EFC40F2026008F088F880230322C0
:103B100010213C4807F0BEFB00228021394807F005
:103B200067FB3949002007F02DF83849002007F0DD
:103B300029F8374806F0D4FD002033490871487150
:103B40008871C871087248720870487004208870C3
:103B50000220C870182048812D4806F05FFE002022
:103B60002A49488188810120C8811B480068000CCF
:103B70000880194800884880012088804FF6FF702F
:103B8000C8800020088101200874084606F0BEFDA8
:103B900001201E49488112480068000C0880104826
:103BA00000884880084606F0B1FD02201749488188
:103BB0000D480068000C08800B48008848800846C3
:103BC00006F0A4FD00F0BCFB0221114806F0BBFE8C
:103BD00010BD0000D20E00209C000020DC0E002052
:103BE000A0000020E60E0020A4000020B40B00205E
:103BF000B40C0020B40D0020F00E0020B40A002008
:103C0000000C014000080140B40E0020C00E00204E
:103C10000064004010B540F2197007F0FFFF40F259
:103C2000036007F0FBFF4FF4C06007F0F7FF4FF4AD
:103C30008073032248213B4807F02CFB4FF40073AC
:103C400003221821374807F025FB01214FF4EA1021
:103C500007F086FB40F2026007F0E0FF80230322BA
:103C60001021314807F016FB002280212E4807F072
:103C7000BFFA2E49002006F085FF2D49002006F0EE
:103C800081FF2C4806F02CFD00202849087148715E
:103C90008871C87108724872087048700420887072
:103CA0000220C87018204881224806F0B7FD002085
:103CB0001F49488188810120C8811F480068000C85
:103CC00008801D4800884880012088804FF6FF70DA
:103CD000C8800020088101200874084606F016FDFF
:103CE00001201349488115480068000C08801348DA
:103CF00000884880084606F009FD02200C494881EA
:103D00000F480068000C08800D480088488008466D
:103D100006F0FCFC00F014FB0221064806F013FE3E
:103D200010BD0000000C014000080140B40E00204E
:103D3000C00E0020006400409C000020A000002075
:103D4000A400002010B506F05BF9034800210170C3
:103D50000020FFF74BF910BD040000202DE9FC5FA7
:103D60004FF0000904F06AF840B1644840786449B3
:103D70000872644840784872002088726048006881
:103D80005F4948605D4890F89400A0B15B48407876
:103D900088B10846007A5949497888420BDD58486D
:103DA000007A56494978401A00F0FF095448807A51
:103DB00048445349887251484078514908725148E3
:103DC00090F89400A0B14F48407888B10846407AF6
:103DD0004C49497888420BDD4948407A494949783D
:103DE000401A00F0FF094648807A484444498872E6
:103DF00044484078424948724048407841494978AF
:103E000008443F49C872B9F1000F44D00846807A8F
:103E1000072840DB08464068B0F52F7F3BD9887AF9
:103E2000FEF787FB0746884635494868FEF781FB61
:103E300082463A464346FEF704FB04460D460022FE
:103E4000314B20462946FEF7B3FB01D200242E4D0C
:103E500000222E4B20462946FEF7C2FB01D2002449
:103E60002A4D2B4A2B4B20462946FEF778FA8246EC
:103E70008B462349D1E90671254A274B3846FEF780
:103E80006EFA52465B46CDE90001FEF7C1F91C4AC5
:103E9000C2E9060100BF1A49C87AFEF74AFB074685
:103EA00088461749D1E9064322464146FEF757FAAC
:103EB00082460022194BFEF7C4FACDE90001FEF755
:103EC0005EFB0646C82E00D9C8260D490E7308466B
:103ED000007B48B10948C07C00F0400020B9094887
:103EE000C07C00F0400030B10448007805490978F2
:103EF000084403490873BDE8FC9F00004007002008
:103F0000A0010020E408002000C0724000E08540CD
:103F10009A9999999999C93F9999E93F00408F4099
:103F200070B5044666680025802229466D1C7254CF
:103F3000522229466D1C72541F48027829466D1C76
:103F400072540088021229466D1C72541B48027874
:103F500029466D1C72540088021229466D1C725449
:103F6000E07820F018001830E070208820F47E708F
:103F700000F506702080B4F8010020F4FE7000F512
:103F80008470A4F80100A07820F03E00801CA0708E
:103F9000681EC11700EB5171C910491C628861F39A
:103FA0008A126280E07820F0E000E07025810E2126
:103FB000204604F0AFFF70BD5A0000205C000020D6
:103FC00070B50446666800BF2D4880782D49497851
:103FD000884200D00FE02A48C0782A49C978884230
:103FE00000D008E0264880882649B1F80D108842A4
:103FF00000D000E070BD00BF2248407820498870A2
:104000002048C078C8701F48B0F80D008880072588
:10401000E07820F018000830E070208820F47E70EE
:1040200000F506702080B4F8010020F4FE7000F561
:104030008470A4F80100A07820F03E00801CA070DD
:10404000681EC11700EB5171C910491C628861F3E9
:104050008A126280E07820F0E000E07025812A4634
:1040600007493046FEF76AF801200749087000202A
:1040700048800021204604F04DFF00BFBAE7000051
:1040800060000020400700206E00002070B504464C
:10409000666800BF2D4880782D494978884200D055
:1040A0000FE02A48C0782A49C978884200D008E041
:1040B000264880882649B1F80D10884200D000E0DB
:1040C00070BD00BF22484078204988702048C078E1
:1040D000C8701F48B0F80D0088800725E07820F0F0
:1040E00018000830E070208820F47E7000F506701B
:1040F0002080B4F8010020F4FE7000F58470A4F86C
:104100000100A07820F03E00801CA070681EC1173E
:1041100000EB5171C910491C628861F38A126280F8
:10412000E07820F0E000E07025812A46074930461B
:10413000FEF704F801200749087000204880052197
:10414000204604F0E7FE00BFBAE70000720000203E
:10415000E40800208000002010B5FFF791FC4FF428
:1041600080713E48FEF703F83D4800210160416040
:1041700001813A483A4948604FF480713948FDF767
:10418000F6FF394800210160416001813548364918
:1041900048604FF480713548FDF7E9FF344800214D
:1041A0000160416001813148314948604FF48071BC
:1041B0003048FDF7DCFF304800210160416001819B
:1041C0002C482D49486040212C48FDF7D0FF2C4851
:1041D000002101604160018128482949486029483F
:1041E000002101608180817143F28110254908809E
:1041F000254800210160818043F282102249088015
:104200002248002101608180817143F281201F4991
:1042100008801F4800210160818043F282201C49F0
:1042200008801C4800210160416081604FF4854096
:1042300018490880184800210160416081604FF4EE
:104240008540154908801548002101604160816062
:104250004FF484401149088010BD0000C0010020C7
:10426000C0020020CA020020CA030020D40300209C
:10427000D4040020DE040020DE050020E805002034
:104280002806002060000020670000207200002047
:10429000790000207C090020880900209409002072
:1042A00070B5044666680C2222492348FDF771FF69
:1042B00000B970BD20481F490A6802604A68426020
:1042C000896881600C25E07820F018000830E070E3
:1042D000208820F47E7000F506702080B4F801007C
:1042E00020F4FE7000F58470A4F80100A07820F09E
:1042F0003E00801CA070681EC11700EB5171C910F0
:10430000491C628861F38A126280E07820F0E00044
:10431000E07025812A4608493046FDF70FFF01204D
:1043200006490870002048800A21204604F0F2FD6A
:1043300000BFBEE7880900207C090020480000205B
:1043400010B500220321132007F0F0F90022032109
:10435000142007F0EBF910BD70B51348007808B9C8
:10436000002070BD1148007820B11148007808B1D4
:104370000020F6E703F024FA10B103F089FA08B937
:104380000020EEE7FEF7EAFD0546FEF7FBFD0446DA
:10439000A54201DB2E1B00E0661B642E01DC012020
:1043A000DFE70020DDE70000050000200E00002010
:1043B0000F00002010B516480078012805D01448D9
:1043C0000078022801D0002010BD1248007828B1E2
:1043D00011480078012801D00020F5E703F0D4F857
:1043E00008B10020F0E703F0EBF910B103F050FA48
:1043F00008B90020E8E709484078022803DB0848AC
:104400004078022801DA0020DEE70120DCE7000026
:10441000050000200E0000200F00002040070020B3
:10442000E408002010B54FF4C06007F0F7FB00224D
:1044300001210A2007F07AF90421022006F0DEFEAD
:1044400002220021102006F0FFFB102006F060FC85
:1044500010BD000010B5002004F0FCFF002007494B
:10446000087007484078642806DB064840786428CE
:1044700002DB01200449087010BD00001D0000206F
:1044800040070020E4080020EC00002010B50024C4
:104490004FF480510B4806F05BFF08B1002010BDBF
:1044A0000948C07C00F0080050B903F08FFA0446B8
:1044B000601C28B104488068A04201D20120EEE7C8
:1044C0000020ECE7000C0140E408002010B50024B7
:1044D0004FF480510B4806F03BFF08B1002010BD9F
:1044E0000948C07C00F0080050B903F06FFA044698
:1044F000601C28B104488068A04201D20120EEE788
:104500000020ECE7000C0140400700202DE9F041BD
:1045100005272C48007840B12B48007828B104F0DA
:104520007BFC07463846BDE8F08103F049F9F8B155
:1045300003F0AEF9E0B12548C07C00F00600062883
:1045400007D00B20214981F88C0003211F48C0F8B7
:1045500090101F48C07C00F0060006280DD00B20EC
:104560001B4981F88C0003211948C0F8901004E021
:1045700004F052FC07463846D5E71448406844F634
:104580002061884203DC12484068884204DD04F060
:1045900043FC07463846C6E7FEF7E0FC0546FEF753
:1045A000F1FC0446A54201DB2E1B00E0661B40F631
:1045B000C410864204DD04F02FFC07463846B2E7FB
:1045C0003846B0E70E0000200F0000204007002012
:1045D000E408002070B505263A48007840B13A4812
:1045E0000078012804D004F017FC0646304670BD60
:1045F0003648007820B104F00FFC06463046F6E756
:1046000002F0C2FF20B104F007FC06463046EEE798
:1046100003F0D6F820B303F03BF908B32C48C07C74
:1046200000F0060006280AD001202A49087004F08C
:10463000F3FB06460020274908703046D7E7264896
:10464000C07C00F0060006280FD001202349087026
:1046500004F0E2FB06460020204908703046C6E719
:1046600004F002FC06463046C1E7FEF777FC05463B
:10467000FEF788FC044644F62060854201DD844252
:1046800008DC1748007840B901201549087000205F
:10469000488002E01248002101601148007878B19A
:1046A0000F484088B0F57A6F0ADB0D4800210160A1
:1046B00004F0B2FB0646012004490870304696E734
:1046C000304694E70E0000200F0000201F0000205D
:1046D000400700201B000020E40800201C000020F0
:1046E0001200002010B5052403F06AF8D8B10F4875
:1046F000C07C00F00600062807D00C48B0F80D007A
:1047000040F60201084000B900240948C07C00F0CE
:104710000A0048B10B20064981F88C0000210448AA
:10472000C0F8901000E00024204610BD4007002093
:10473000E408002010B5052403F0AAF8D8B10F480A
:10474000C07C00F00600062807D00C48B0F80D0029
:1047500040F60201084000B900240948C07C00F07E
:104760000A0048B10B20064981F88C00002104485A
:10477000C0F8901000E00024204610BDE40800209E
:104780004007002010B5052404F0B6FE10B104F077
:10479000E7FE00B910BD1B480078052818D2DFE8F5
:1047A00000F003070B0F130004F036FB044610E083
:1047B000FFF798FF04460CE0FFF7BCFF044608E053
:1047C000FFF7A4FE044604E0FFF704FF044600E000
:1047D000E0E700BF052C07DB0B48007818B9032180
:1047E000012003F0D5F9D5E73CB907480078012846
:1047F00003D10121002003F0CBF92046FEF7F6FBA0
:1048000000BFC7E7050000200D00002010B50D48CF
:104810000078B0B10C4805F073FF90B1012211038C
:104820000A4806F0E5FC084805F05AFFFFF7F2F9E0
:1048300000224FF48051054806F0DAFC00200449BC
:10484000087010BD0D000020006400400008014009
:10485000A800002010B50548FFF7B2FB0448FFF799
:1048600015FC0448FFF71CFD10BD0000CA03002022
:10487000D4040020DE05002010B55048407861289F
:1048800003DB4F484078612802DA00204D49087068
:1048900002F07AFE00286ED04B48007828B3002042
:1048A0004A4908704A48007804280AD10320FFF7D3
:1048B00047F8032822D101221103464806F098FC4C
:1048C0001CE001221103434806F092FC40480078A6
:1048D000012803D03E48007802280FD13E480078D6
:1048E00060B901203C49087008E039480078042884
:1048F00004D001221103374806F07AFC4FF48051AE
:10490000344806F025FD002857D02C48C078B8B9A7
:104910002B48C078A0B93148007828B901202F4928
:104920000870002048800EE02C48408842F2107148
:10493000884208DB294800210160FFF78BFD02E077
:1049400026480021016022480078032835D11B4801
:10495000C07888B11A48407B00F02000F8B11748B1
:10496000406817494968084441F28831884224DA8E
:10497000FFF770FD21E013E01148C07878B10F48CF
:10498000407B00F0200050B10C4840680C49496859
:10499000084441F2883188420FDAFFF75BFD0CE0F2
:1049A00000224FF480510B4806F022FC06480078A4
:1049B00018B10B4800780549087010BD4007002069
:1049C000E4080020EC0000200E0000200F00002072
:1049D00005000020000C01401D000020E000002028
:1049E000100000200448007820B103484088401C93
:1049F0000149488070470000E000002010B574486D
:104A00000078A8B172484088642811DB7048002102
:104A100001604FF480616F4806F092FC08B90120F4
:104A200000E000206C49C97860F3C3016A48C17096
:104A30006A484078B8B169484088B0F5FA6F12DB2F
:104A400000206649487048804FF40061614806F0D4
:104A500077FC08B9012000E000205F49C97860F3C5
:104A6000C7115D48C1705E480078A8B15C484088B5
:104A7000642811DB5A48002101604FF480515548E9
:104A800006F05EFC08B9012000E000205249C97818
:104A900060F304115048C1705248007830B1514859
:104AA0004088642802DB4F48002101604E480078AE
:104AB000A0B14D484088642810DB4B4800210160BC
:104AC00040214A4806F03CFC08B9012000E00020E3
:104AD0004149C97860F300013F48C17044480078FB
:104AE000C0B143484088642814DB00204049488016
:104AF0004048007858B94048006808B1012000E0FB
:104B000000203549C97860F382013348C170002024
:104B10003949086039480078A0B13848408864288D
:104B200010DB3648002101600121354806F008FC01
:104B300008B9012000E000202749097960F300014D
:104B40002548017102F020FD2349097960F34101F4
:104B5000214801712B4840781F4948712948007845
:104B6000887129480078C871284800780872284858
:104B7000007848722748D0E906211046FDF7FFFC6F
:104B80001549488124480A6802604A684260896879
:104B900081601021154806F0DBFB1F49C97860F3DE
:104BA00041011D48C1700221104806F0D1FB1A498D
:104BB000C97860F345111848C17001210B4806F00F
:104BC000C7FB1549C97860F386111348C17010BD41
:104BD000B80000200010014088090020E4000020F7
:104BE000BC000020C0000020C4000020000C0140D8
:104BF000C8000020DC000020E8000020CC000020DD
:104C00000014014044000020310000203A00002040
:104C100005000020A00100209409002010B50948DB
:104C2000006800048209A2F5805000F100610B8841
:104C3000088842F22334A04201D1012010BD002097
:104C4000FCE70000E0F7FF1F70B504460D4634B1E5
:104C500004F026F800B3012004F00EF81CE004F084
:104C60001FF8C8B115B1012D14D106E0FDF734FECF
:104C700010B9002004F000F80DE04021074806F0CC
:104C80005FFB08B9012000E0002010B9002003F00C
:104C9000F3FF00E070BD00BF00BFFBE7000C014068
:104CA00010B54021084806F04BFB08B9012000E090
:104CB000002040B9FDF710FE28B903F0F1FF10B154
:104CC000002003F0D9FF10BD000C01402DE9F04198
:104CD0001A48006800048609A6F5006000F1006427
:104CE000002543F230072068401C30B112222146D3
:104CF0001348FDF723FABDE8F08106F071F900F0E2
:104D000043FB204606F0F6F8002507E000F03CFBE8
:104D10006019394606F078F8A81CC5B2122DF5DBEB
:104D200006F0D2F8A6F5006000F1006412222146D8
:104D30000348FDF703FA00BFDDE70000E0F7FF1FBF
:104D40000401002010B503F0BDFF58B1104890F8E1
:104D50009400E0B901200E4981F89400052081F803
:104D60008C0014E00A4890F8940080B1982108481B
:104D7000FDF7FDF9074800210160416081600020D6
:104D8000054908700520024981F88C0000BF10BD5C
:104D900040070020340700203000002010B503F049
:104DA00097FF58B1104890F89400E0B901200E49DF
:104DB00081F89400052081F88C0014E00A4890F8EE
:104DC000940080B198210848FDF7D1F907480021E7
:104DD000016041608160002005490870052002499A
:104DE00081F88C0000BF10BDE4080020D808002026
:104DF0003900002010B5012005F090FF38B10120E6
:104E000005F086FF0120024908700020488010BD8F
:104E1000CC00002010B54FF4806005F07FFF40B15A
:104E20004FF4806005F074FF0120244908700020D1
:104E300048804FF4006005F071FF58B14FF40060F6
:104E400005F066FF1E48007820B101201C4948701B
:104E5000002048804FF4805005F060FF40B14FF4CF
:104E6000805005F055FF0120164908700020488049
:104E70004FF4005005F052FF18B14FF4005005F008
:104E800047FF4FF4804005F049FF60B14FF4804088
:104E900005F03EFF0C48007818B101200B4908705E
:104EA00010BDFDF7C3FC4FF4004005F037FF18B10B
:104EB0004FF4004005F02CFF00BFF1E7B8000020E0
:104EC000E4000020BC0000208400002086000020B8
:104ED00010B5022005F022FF10B1022005F018FFE6
:104EE00010BD10B5082005F019FF10B1082005F01D
:104EF0000FFF10BD10B5102005F010FF50B11020AD
:104F000005F006FF1021044806F01AFA10B9012036
:104F100004F0A0FA10BD00000010014010B52020E0
:104F200005F0FCFE10B1202005F0F2FE402005F057
:104F3000F5FE38B1402005F0EBFE0120164908705F
:104F400000204880802005F0E9FE70B1802005F047
:104F5000DFFE1248007828B911480068401C10494B
:104F6000086002E000200E4908604FF4807005F0F0
:104F7000D5FE28B14FF4807005F0CAFEFDF768FD3C
:104F80004FF4007005F0CAFE28B14FF4007005F030
:104F9000BFFEFDF737FE10BDC4000020DC0000207E
:104FA000E800002010B54FF4C06006F037FE002284
:104FB0000121282006F0BAFB0A21022006F01EF982
:104FC00002220021500205F03FFE4FF4806005F000
:104FD0009FFE0B21022006F011F90222002190020F
:104FE00005F032FE4FF4006005F092FE0C21022025
:104FF00006F004F902220021D00205F025FE4FF44C
:10500000805005F085FE0E21022006F0F7F80122FF
:105010000021900305F018FE4FF4804005F078FE63
:1050200000220121172006F081FB0621012006F055
:10503000E5F802220021402005F006FE402005F0A0
:1050400067FE00220121062006F070FB00210320EC
:1050500006F0D4F802220021012005F0F5FD012020
:1050600005F056FE0721012006F0C8F801220021B4
:10507000802005F0E9FD802005F04AFE10BD00000B
:1050800010B540F2046006F0C9FD4FF4004303225E
:105090001021494806F0FEF80020FDF7FBFB4FF415
:1050A000804303224821444806F0F4F840F20560AA
:1050B00006F0B4FD4FF4C06006F0B0FD0121C80356
:1050C00006F04EF90123032248213C4806F0E2F89D
:1050D000C02303221021384806F0DCF800224021CA
:1050E000354806F085F800228021334806F080F824
:1050F00040F2036006F092FD03231A461021304867
:1051000006F0C8F8002201212D4806F071F80022AF
:1051100002212B4806F06CF84FF47053032248210B
:10512000254806F0B7F840F2036006F077FD30231B
:1051300003221021224806F0ADF800221021204859
:1051400006F056F80521002002F064FDC02303227A
:1051500048211B4806F09EF8FFF724FF012019495B
:1051600008706420488001201749087048704FF487
:10517000FA604880012015490870642048800120A9
:105180001349087064204880012012490870642087
:1051900048800120104908706420488001200F4990
:1051A0000870642048800E48002101600D480160AD
:1051B0000D48016010BD00000010014000140140C6
:1051C000000C0140B8000020E4000020BC000020DA
:1051D000C0000020C4000020C8000020CC00002037
:1051E000D4000020D8000020DC00002028B10122DB
:1051F000044B1A701A46518002E0024A00231360E1
:1052000070470000B400002028B10122044B1A703E
:105210001A46518002E0024A0023136070470000E2
:10522000F800002010B5FFF72BFF88210148FCF79C
:105230009EFF10BD180100201848007848B3174899
:105240004088401C1549488008464088B0F5967F44
:1052500009DB0846002101601148006840F48040E5
:105260000F49086018E00D484088C82806D10C484E
:10527000006840F480400A4908600DE00748408813
:10528000642809D10648006840F480400449086059
:1052900002E00020014948807047000048000020DB
:1052A0000000002006F0CAFD234807F0D3F8234889
:1052B00007F0D0F8224805F013FA02F057FD00BFBE
:1052C00040F21C7006F0AAFC0021012006F098FABA
:1052D00004F006FB06F0C0FD02F042FB02F076FB94
:1052E000044606F0ABFD44F62060844223D91548FD
:1052F000844220D2012080F3138800BF00BF00BF8A
:1053000000BF00BF00BFBFF34F8F00BF00BF00BF93
:105310000D48006800F4E0600C490843001D0A498C
:10532000086000BF00BF00BFBFF34F8F00BF00BFCA
:1053300000BF00BFFEE7C3E7003801400044004063
:1053400000640040C0D401000CED00E00000FA054C
:105350000B48007890B10A484088401C80B2084948
:10536000488043F69821884208DB05480021016007
:105370000448006840F400100249086070470000CB
:105380008C0000200000002010B540F2073005F02E
:105390002BFD10BD10B540F2026006F03FFC40F25C
:1053A000036006F03BFC40F2046006F037FC4FF46B
:1053B000C06006F033FC012303224821224805F097
:1053C00069FF0623032248211F4805F063FF4FF4BD
:1053D0008053032210211D4805F05CFF01221103B8
:1053E0001A4805F005FF0121194805F0B9FF4FF4EF
:1053F000004303224821154805F04CFF08230322EF
:105400001021144805F046FF00220821114805F03C
:10541000EFFE1023032248210B4805F03BFF4FF419
:105420008053032210210B4805F034FFFEF7FAFFEA
:10543000042303221021074805F02CFF0122042138
:10544000044805F0D5FE10BD0010014000080140E1
:1054500000023000000C014010B504460B460CB1B0
:1054600003B10AB9002010BD002104E018880144EE
:105470009B1C901E82B2012AF8DC002A01DD1878FC
:10548000014402E088B200EB1141080C0028F9D178
:10549000C84320800120E6E710B504460B460CB156
:1054A00003B10AB9002010BD002104E018880144AE
:1054B0009B1C901E82B2012AF8DC002A01DD1878BC
:1054C000014402E088B200EB1141080C0028F9D138
:1054D000C84320800120E6E770B5044600250CB9DA
:1054E000002070BD30488078C0F3440020B12E48C1
:1054F0008078C0F3440000E0202070B12A48807812
:10550000C0F3440028494988C1F38411884204D17A
:105510002548008908B1244D34E024488078C0F340
:10552000440020B121488078C0F3440000E02020EE
:1055300070B11E488078C0F344001C494988C1F30B
:105540008411884204D11948008908B1174D19E027
:1055500017488078C0F3440020B115488078C0F324
:10556000440000E0202068B111488078C0F3440076
:105570000F494988C1F38411884203D10C4800893E
:1055800000B10B4D0DB90020ABE7286820602A89D7
:1055900069686068FCF7D2FD28892081284602F0FE
:1055A00069FC20899DE70000D20E0020DC0E00205F
:1055B000E60E00200248C07800F0010070470000AD
:1055C0008809002070B505460C461DB108480088C2
:1055D000844201DA002070BD05480288054928464A
:1055E000FCF7ACFD0248048802F062FC2046F2E7BA
:1055F000F20000200C12002070B505460C461DB1CB
:1056000008480088844201DA002070BD05480288FD
:1056100005492846FCF792FD0248048802F03AFC4E
:105620002046F2E7AE000020FA0F002010B540F24D
:10563000073005F0D9FB10BD10B502460B4600201F
:10564000002104E0545C0444E0B24C1CE1B29942F5
:10565000F8DB10BD70B50446264600BF0CB900202B
:1056600070BDB078012800D06FE0F5780020F070B0
:1056700031782046FFF7E0FFA84200D065E004251E
:1056800070780D285CD2DFE800F0070D223D525300
:105690005455565758595A000122D1032C4805F049
:1056A000A7FD4FE0605D012805D1012208212848AF
:1056B00005F09EFD0AE0605D022805D10022082168
:1056C000234805F095FD01E00020C9E73AE0605D60
:1056D000012808D1002201031E4805F089FD0120A0
:1056E0001D4908700DE0605D022808D10122C10249
:1056F000184805F07DFD00201749087001E00020E2
:10570000AEE71FE0605D012805D10122202110488D
:1057100005F06EFD0AE0605D022805D1002220211F
:105720000B4805F065FD01E0002099E70AE009E07B
:1057300008E007E006E005E004E003E002E001E045
:1057400000208DE700BF01208AE700BF002087E727
:10575000000C0140000801400D00002070B5044617
:1057600034B94FF480711B48FFF746FFC5B209E01A
:10577000012C05D121021748FFF724FFC5B201E033
:10578000002070BD1448047012480078A84201D06F
:105790000020F6E70F48FFF75DFF08B90020F0E7AB
:1057A0000C4800F0B1F808B90020EAE734B909481C
:1057B000017803F00BFC50B90020E2E7012C06D180
:1057C0000448017803F082FB08B90020D9E70120E2
:1057D000D7E70000B40900208500002010B54FF481
:1057E0000051364805F0ACFD18B1FFF717FA00B9C3
:1057F00010BD334806F07CF8002004F097FB012030
:105800003049087030480021016000BFFEF7FEFFFC
:1058100000F0EAFE2D48007800F0010040B10020C1
:10582000FFF79CFF2948006820F001002749086025
:105830002648007800F0040040B10120FFF78EFFF9
:105840002248006820F00400204908601F480068D2
:1058500000F4803038B1FDF77FF91C48006820F46F
:1058600080301A4908601948006800F4003038B1E7
:10587000FDF792F91548006820F4003013490860DC
:105880001248006800F4802048B1FDF7C5F8FDF724
:10589000A5F90E48006820F480200C4908600B48E8
:1058A000006800F400200028B0D0FDF7C3F80748D6
:1058B000006820F4002005490860A7E700100140B7
:1058C00044332211840000202C000020000000201E
:1058D0000B48007890B10A484088401C80B20849C3
:1058E000488040F6B831884208DD05480021016053
:1058F0000448006840F480000249086070470000D6
:1059000088000020000000202DE9F04105462E46C9
:1059100015B90020BDE8F08170780D2877D2DFE856
:1059200000F0070D1319277AF1F0EFEEEDECEB0024
:10593000042400222146641C6A548CE304240022BF
:105940002146641C6A5486E3042400222146641C18
:105950006A5480E304244021FA4805F0F1FC08B1C0
:10596000012200E000222046611CCCB22A5472E3DE
:105970000424285D01280AD100220421F14805F001
:1059800037FC00222046611CCCB22A5442E0285D3C
:10599000022810D10020EC4908700122D103EB4805
:1059A00005F026FC0121EA4805F0CAFC2146621CEC
:1059B000D4B268542EE0285D032809D1E248027869
:1059C0002046611CCCB22A540020DF49087021E037
:1059D000285D04280DD100224103DC4805F008FCB5
:1059E0000121DB4805F0ACFC2146621CD4B26854AE
:1059F00010E0285D05280BD101220421D14805F0D3
:105A0000F7FB00222046611CCCB22A5402E021E3BD
:105A100000207FE71FE30424285D01283AD10022FB
:105A20004103C84805F0E4FB00226103C54805F0C6
:105A3000DFFB00222103C34805F0DAFB642005F0F8
:105A4000F1F80221C14805F07BFC2146621CD4B26A
:105A500068540421BD4805F073FC2146621CD4B291
:105A6000685401F0B3FF07462046611CCCB22F54A6
:105A7000C7F307222046611CCCB22A54C7F3074261
:105A80002046611CCCB22A543A0E2046611CCCB28E
:105A90002A547EE1285D022845D1601C285C01283B
:105AA0000AD10122C103A74805F0A2FB002220462B
:105AB000611CCCB22A546CE1601C285C022822D103
:105AC000642005F0AFF801F081FF07462046611C15
:105AD000CCB22F54C7F307222046611CCCB22A5403
:105AE000C7F307422046611CCCB22A543A0E204626
:105AF000611CCCB22A544CE17FE268E241E20CE244
:105B0000EBE1A2E146E1601C285C0328C1D1002240
:105B10004FF400418B4805F06BFB00222046611CCE
:105B2000CCB22A5435E1285D03282BD1642005F03E
:105B300079F80221854805F003FC2146621CD4B2A5
:105B400068540421814805F0FBFB2146621CD4B255
:105B5000685401F03BFF07462046611CCCB22F542D
:105B6000C7F307222046611CCCB22A54C7F3074270
:105B70002046611CCCB22A543A0E2046611CCCB29D
:105B80002A5406E1285D04284BD1601C285C0128BA
:105B900012D1002204216B4805F02AFB0A2005F0EF
:105BA00041F801225103674805F022FB00222046FC
:105BB000611CCCB22A54ECE0601C285C02281BD18A
:105BC000642005F02FF801F001FF07462046611C14
:105BD000CCB22F54C7F307222046611CCCB22A5402
:105BE000C7F307422046611CCCB22A543A0E204625
:105BF000611CCCB22A54CCE0601C285C032891D1F3
:105C0000012204214F4805F0F3FA00224FF400511D
:105C10004C4805F0EDFA00222046611CCCB22A5413
:105C2000B7E0285D05282BD1642004F0FBFF02219A
:105C3000464805F085FB2146621CD4B26854042115
:105C4000424805F07DFB2146621CD4B2685401F045
:105C5000BDFE07462046611CCCB22F54C7F3072275
:105C60002046611CCCB22A54C7F307422046611C6F
:105C7000CCB22A543A0E2046611CCCB22A5488E099
:105C8000285D06283ED1601C285C01280AD101222B
:105C900081032C4805F0ACFA00222046611CCCB2EE
:105CA0002A5476E0601C285C02281BD1642004F092
:105CB000B9FF01F08BFE07462046611CCCB22F5481
:105CC000C7F307222046611CCCB22A54C7F307420F
:105CD0002046611CCCB22A543A0E2046611CCCB23C
:105CE0002A5456E0601C285C032852D100224FF44D
:105CF0008041144805F07CFA00222046611CCCB299
:105D00002A5446E0285D072824D1002204210D48AA
:105D100005F06EFA0A2004F085FF012251030948BC
:105D200005F066FA0122D103064805F061FA012266
:105D30009103044805F05CFA00222046611CCCB2B5
:105D40002A5426E0000C014086000020001001408B
:105D500000140140285D08280AD10022C102C4486D
:105D600005F046FA00222046611CCCB22A5410E00D
:105D7000285D09280BD100224FF40041BC4805F0F2
:105D800037FA00222046611CCCB22A5401E00020E0
:105D9000C0E560E10424285D012819D1002280219A
:105DA000B44805F025FA00220121B14805F020FA97
:105DB00001224021AF4805F01BFA01220221AC4824
:105DC00005F016FA00222046611CCCB22A543BE0B2
:105DD000285D022819D100224021A64805F008FAC2
:105DE00000220221A24805F003FA01228021A148E5
:105DF00005F0FEF9012211469D4805F0F9F900224F
:105E00002046611CCCB22A541EE0285D032819D11B
:105E100000228021974805F0EBF9002201219448E7
:105E200005F0E6F900224021924805F0E1F9002250
:105E300002218F4805F0DCF900222046611CCCB21B
:105E40002A5401E0002065E505E10424285D0128CD
:105E50001ED18102874805F073FA2146621CD4B234
:105E600068544FF40061834805F06AFA08B10122D2
:105E700000E000222046611CCCB22A544FF480512D
:105E80007C4805F05DFA2146621CD4B2685423E0D8
:105E9000285D02281ED14102764805F051FA2146BC
:105EA000621CD4B268544FF40061724805F048FA9D
:105EB00008B1012200E000222046611CCCB22A5425
:105EC0004FF480516B4805F03BFA2146621CD4B276
:105ED000685401E000201DE5BDE00424285D012890
:105EE0000AD101221021624805F082F900222146E0
:105EF000601CC4B26A540FE0285D02280AD1002257
:105F000010215B4805F074F900222046611CCCB2D8
:105F10002A5401E00020FDE49DE00424285D0128CE
:105F200014D1002054490860642004F07BFE5248DC
:105F3000006828B101222046611CCCB22A541FE01F
:105F400000222046611CCCB22A5419E0285D0228A8
:105F500014D1002048490860642004F063FE4648DC
:105F6000006828B101222046611CCCB22A5407E007
:105F700000222146601CC4B26A5401E00020C9E43A
:105F800069E00424285D01280DD10122010338486D
:105F900005F02EF91021374805F0D2F92146621C90
:105FA000D4B2685412E0285D02280DD10022C1024B
:105FB0002F4805F01DF910212E4805F0C1F92146A2
:105FC000621CD4B2685401E00020A3E443E004243E
:105FD000285D01280ED105F0AFF828480278204648
:105FE000611CCCB22A54254842782046611CCCB2B0
:105FF0002A5401E000208DE42DE00424285D0128CE
:1060000007D1FCF7E1FC00222046611CCCB22A54E7
:106010001FE0285D02281AD1194802782046611C29
:10602000CCB22A541648008802122046611CCCB219
:106030002A54144802782046611CCCB22A541148D4
:10604000008802122046611CCCB22A5401E00020D4
:1060500060E400E000BF00BF34700020B070F0705A
:1060600031782846FFF7E8FAF070012052E400008A
:10607000000C014000100140E80000204400002016
:106080005A0000205C00002008B5014648680088DE
:106090000090BDF8000043F20D13C21A984225D0BB
:1060A00013DC43F20613A0EB030298421DD007DC79
:1060B000B0F5445F16D0A0F54450053800BB12E09F
:1060C000012A15D0062A1BD10EE0032A12D004DCC7
:1060D000012A0CD0022A13D10BE0042A0BD0742A17
:1060E0000ED109E00EE00DE00CE00BE00AE009E063
:1060F00008E007E006E005E00020044A107008BD53
:106100000020FCE700BF0120F9E700006E0000203E
:1061100008B50146486800880090BDF8000043F2C9
:106120000D23C21A984225D013DC43F20623A0EBBC
:10613000030298421DD007DCB0F5485F16D0A0F5E9
:106140004850053800BB12E0012A15D0062A1BD1A1
:106150000EE0032A12D004DC012A0CD0022A13D14B
:106160000BE0042A0BD0742A0ED109E00EE00DE0FA
:106170000CE00BE00AE009E008E007E006E005E0DB
:106180000020044A107008BD0020FCE700BF012079
:10619000F9E700008000002070B50446606845788B
:1061A000432D40D006DC312D09D0322D20D0422D98
:1061B0005FD137E0482D34D0522D5AD14CE02F48D2
:1061C0002168016020892D4908810B461A89616880
:1061D0005868FBF7B3FF2948FFF756FF08B90020BE
:1061E00070BD264801F072FE08B90020F8E741E0D2
:1061F0002348216801602089214908810B461A89BA
:1062000061685868FBF79AFF1D48FFF781FF08B9DE
:106210000020E5E71A4802F037F808B90020DFE768
:1062200028E000BF00BF1748216801602089154998
:1062300008810B461A8961685868FBF77FFF11488F
:1062400000F024F808B90020CAE70E4802F0F2F97D
:1062500008B90020C4E70DE00B48216801602089DF
:10626000094908810B461A8961685868FBF766FF7F
:1062700000E000BF00BF0120B2E70000CA03002019
:10628000D4040020DE0500202806002038B505468D
:106290006C68686800880090BDF8000044F2F02245
:1062A000811A904272D01EDC44F20622A0EB020159
:1062B000904255D008DCA0F58440062867D2DFE87C
:1062C00000F03238393D4D4E042950D006DC01290A
:1062D0004AD0022949D0032959D147E005294BD09A
:1062E0007A29F9D157E1152971D00EDC112944D052
:1062F00006DC05296CD006296BD00829ECD152E1C7
:1063000012295FD01329E7D177E0182970D004DC77
:1063100016296ED01729DFD11AE128296AD0B1F5E4
:10632000A26FD9D136E1A07800F00100A149087030
:106330003CE13BE1A078A049087037E1A078012852
:1063400002D19E49087008E0A078022803D10020FD
:106350009A49087001E0002038BD27E126E125E1D7
:10636000A01C03F011FE21E120E11FE11EE1944891
:10637000D4F80210016019E118E192480078012870
:106380001FD1A07820B1012815D109E007E10BE168
:106390000221002001F03EFC00208B4908700CE037
:1063A0000321012001F036FCFCF796FA10B9012018
:1063B000FCF770FA01E00020CEE700BF0A2004F0ED
:1063C00031FCF3E0A07828B101280FD108E071E09A
:1063D000E7E0E7E0002210217C4804F009FF0AE032
:1063E00001221021794804F003FF04E00020B3E704
:1063F000B9E089E073E000BFD8E0A07840B900229E
:106400004021734804F0F4FE00207249087048806F
:10641000A078012804D1012240216D4804F0E8FE53
:10642000A078022809D101224021694804F0E0FE49
:1064300001206849087000204880A07803280AD10C
:1064400000224021624804F0D3FE01206149087017
:106450004FF416704880E07840B9002280215C48F3
:1064600004F0C6FE00205C4908704880E0780128EE
:1064700004D101228021564804F0BAFEE0780228B7
:1064800009D101228021524804F0B2FE0120524974
:10649000087000204880E07803280AD1002280217B
:1064A0004B4804F0A5FE01204B4908704FF41670CC
:1064B00048807BE0A07810B101280CD105E00022D3
:1064C0000221424804F094FE07E0012202213F48E5
:1064D00004F08EFE01E000203EE700BF66E0A078F9
:1064E00010B101280CD105E000220121374804F049
:1064F0007FFE07E001221146344804F079FE01E0F6
:10650000002029E700BF51E02E48007801281ED165
:10651000A07810B1012814D10CE040212B4804F0E0
:106520000FFF08B9012000E0002010B90020FCF79F
:10653000B1F908E0FCF7D0F910B90120FCF7AAF98D
:1065400001E0002008E700BF0A2004F06BFB2DE00B
:106550001C480078012805D1A07820490870E0780F
:106560001F49087022E0A07810B101280BD103E088
:106570000020FCF78FF908E0FCF7AEF910B9012014
:10658000FCF788F901E00020E6E600BF0A2004F0ED
:1065900049FB0BE00AE0002012490870DCE605F038
:1065A0007DF900BF00BF01E00020D5E600BF01205B
:1065B000D2E60000E40000200E00002010000020C1
:1065C000A00100200D0000201F000020000C014051
:1065D00000100140D4000020D80000203600002028
:1065E0003E0000204800002070B5B848FEF774FF58
:1065F000C4B20CB9002070BDB548007801287DD127
:10660000B4480078FF28FAD1B2484078FF28F6D184
:1066100002242146641CAF48405CAF49087008461C
:10662000007810286BD008DCA0F10A00062867D299
:10663000DFE800F0121CC5F4F3F214287ED006DC6B
:1066400011287CD012287BD0132859D1B8E33028E8
:1066500077D03128F9D1BBE39E49085DFCF7C6FC31
:10666000054629469DA003F007FDB3E39E48017847
:106670009EA003F001FDA34890F89410A2A003F09F
:10668000FBFCA04890F89510A5A003F0F5FC9D48F0
:106690000178A9A003F0F0FC9A484178AAA003F081
:1066A000EBFC98488178ADA003F0E6FC9548C178F2
:1066B000AEA003F0E1FC93484168B1A003F0DCFC1C
:1066C00090488168B3A003F0D7FC8E48017BB7A047
:1066D00003F0D2FC8B48B0F80D10B8A003F0CCFC4E
:1066E0008848D0F80F10BAA003F0C6FC8548C17CDA
:1066F000BDA003F0C1FC1222824902E06DE35CE31D
:1067000067E315317348FBF719FD00207149887460
:10671000BAA003F0B1FC14227A4927316D48FBF787
:106720000DFD00206B490875B7A003F0A5FC754866
:10673000B0F83B10B8A003F09FFC03E041E33DE359
:106740003DE344E36F48D0F83D10B7A003F094FC5C
:106750006C48D0F84110B9A003F08EFC6948D0F81D
:106760004510BCA003F088FC6648D0F84910BFA0D3
:1067700003F082FC6348D0F84D10C3A003F07CFC0A
:106780006048D0F85110C7A003F076FC5D48D0F8FF
:106790005510C9A003F070FC5A48D0F85910CCA08D
:1067A00003F06AFC5748D0F85D10CFA003F064FCFA
:1067B0005448D0F86110D2A003F05EFC0AE3D6483A
:1067C0000178D6A003F058FCDA4890F89410DAA0CB
:1067D00003F052FCD74890F89510DDA003F04CFC74
:1067E000D4480178E0A003F047FCD2484178E2A009
:1067F00003F042FCCF488178E4A003F03DFCCD4893
:10680000C178E6A003F038FCCA484168E8A003F06C
:1068100033FCC848816802E0B4E298E279E2E9A07A
:1068200003F02AFCC348017BECA003F025FCC1481F
:10683000B0F80D10EDA003F01FFCBE48D0F80F100B
:10684000EFA003F019FCBB48C17CF3A003F014FCDB
:106850001222B84915311F48FBF770FC00201D4972
:106860008874F2A003F008FC1422B24927311948B9
:10687000FBF764FC002017490875EFA003F0FCFB50
:10688000AC48B0F83B10F0A003F0F6FBA948D0F8F4
:106890003D10F1A003F0F0FBA648D0F84110F3A0A2
:1068A00003F0EAFBA348D0F84510F6A003F0E4FBA0
:1068B000A048D0F84910F9A003F0DEFB9D48D0F8BD
:1068C0004D10FDA003F0D8FB04E20000C002002040
:1068D00027000020C0010020280000207265747588
:1068E000726E3A25640D0A00310000207375625FF4
:1068F000626D735F315F6C745F73746174653A25A8
:10690000640D0A004007002072733438355F636FEE
:106910006E6E6563745F313A25640D0A00000000F5
:1069200072733438355F74696D655F6F75745F318C
:106930003A25640D0A000000796A6B78736C635F16
:10694000313A25640D0A00006D5F70657263656EF3
:10695000745F313A25640D0A00000000796A6364AF
:106960007763736A5F313A25640D0A006368617268
:1069700067655F666C61675F313A25640D0A0000E8
:106980006D5F63757272656E745F313A25646D6117
:106990000D0A00006D5F746F74616C5F766F6C5FE1
:1069A000313A25756D760D0A00000000626D735F47
:1069B00074656D705F313A25640D0A00776F726BF4
:1069C0005F7374617475735F313A25780D0A000046
:1069D00062616E6C616E63655F63656C6C5F313ABA
:1069E00025780D0A00000000626D735F7374617496
:1069F00075735F313A25780D0A000000736E5F31C0
:106A00003A25730D0A000000736F66745F76657235
:106A10005F313A25730D0A006463736D78735F31DB
:106A20003A25640D0A0000004368617267655F4E95
:106A3000756D5F313A256C750D0A00004F7643681D
:106A40005F766F6C5F4E756D5F313A256C750D0A20
:106A5000000000004F764469735F766F6C5F4E757F
:106A60006D5F313A256C750D0A0000004F76436862
:106A7000617267655F6375725F4E756D5F313A2550
:106A80006C750D0A000000004F76446973636861FD
:106A90007267655F6375725F4E756D5F313A256C25
:106AA000750D0A0053686F72745F4E756D5F313AF1
:106AB000256C750D0A000000556454656D706543C2
:106AC000685F4E756D5F313A256C750D0A000000E8
:106AD000556454656D70654469735F4E756D5F31C3
:106AE0003A256C750D0A00004F7654656D7065434C
:106AF000685F4E756D5F313A256C750D0A000000B8
:106B00004F7654656D70654469735F4E756D5F3186
:106B10003A256C750D0A00003A0000207375625F1B
:106B2000626D735F325F6C745F73746174653A2574
:106B3000640D0A00E408002072733438355F636F17
:106B40006E6E6563745F323A25640D0A00000000C2
:106B500072733438355F74696D655F6F75745F3259
:106B60003A25640D0A000000796A6B78736C635FE4
:106B7000323A25640D0A00006D5F70657263656EC0
:106B8000745F323A25640D0A00000000796A63647C
:106B90007763736A5F323A25640D0A006368617235
:106BA00067655F666C61675F323A25640D0A0000B5
:106BB0006D5F63757272656E745F323A25646D61E4
:106BC0000D0A00006D5F746F74616C5F766F6C5FAF
:106BD000323A25756D760D0A00000000626D735F14
:106BE00074656D705F323A25640D0A00776F726BC1
:106BF0005F7374617475735F323A25780D0A000013
:106C000062616E6C616E63655F63656C6C5F323A86
:106C100025780D0A00000000626D735F7374617463
:106C200075735F323A25780D0A000000736E5F328B
:106C30003A25730D0A000000736F66745F76657203
:106C40005F323A25730D0A006463736D78735F32A7
:106C50003A25640D0A0000004368617267655F4E63
:106C6000756D5F323A256C750D0A00004F764368EA
:106C70005F766F6C5F4E756D5F323A256C750D0AED
:106C8000000000004F764469735F766F6C5F4E754D
:106C90006D5F323A256C750D0A0000004F7643682F
:106CA000617267655F6375725F4E756D5F323A251D
:106CB0006C750D0A000000004F76446973636861CB
:106CC0007267655F6375725F4E756D5F323A256CF2
:106CD000750D0A008948D0F8511089A003F0CCF94D
:106CE0008648D0F855108BA003F0C6F98348D0F839
:106CF00059108EA003F0C0F98048D0F85D1091A023
:106D000003F0BAF97D48D0F8611094A003F0B4F90B
:106D100060E0984890F9001097A003F0ADF995480D
:106D200090F901109AA003F0A7F900F04FFE054674
:106D300029469DA003F0A0F9A0480178A0A003F087
:106D40009BF9A4480178A4A003F096F942E0A84872
:106D5000005D40B10B20A74981F88C000321A548B4
:106D6000C0F8901007E00B20A24981F88C000021A8
:106D7000A048C0F890109F48D0F890109EA003F053
:106D80007BF927E09A48005D40B10B205B4981F810
:106D90008C0003215948C0F8901007E00B20574998
:106DA00081F88C0000215548C0F890105348D0F865
:106DB000901094A003F060F90CE00BE00AE009E009
:106DC00008E09348017893A003F056F902E001E04F
:106DD00000E000BF00BF01200DE4042290A1844820
:106DE000FBF7D7F9002854D104228FA18048001D59
:106DF000FBF7CFF930B90120854908708CA003F06A
:106E00003BF944E008228EA17948001DFBF7C1F947
:106E100030B904207E4908708CA003F02DF936E0CB
:106E200006228FA17248001DFBF7B3F930B902208A
:106E3000774908708CA003F01FF928E005228EA185
:106E40006B48001DFBF7A5F930B9032070490870A5
:106E50008BA003F011F91AE006228DA16448001DF1
:106E6000FBF797F930B90020694908708AA003F050
:106E700003F90CE005228CA15D48001DFBF789F9A0
:106E800018B98BA003F0F8F801E00020A4E7012076
:106E9000A2E75F480078022807D155480078FC280F
:106EA00003D153484078FC281FD059480078032864
:106EB00007D14F480078FE2803D14D484078FE287E
:106EC00013D053480078042807D149480078FD289A
:106ED00003D147484078FD2807D000204C4908706E
:106EE0007748FFF759F9012076E71221744802F03C
:106EF00011F808B900206FE701206DE7E4080020D1
:106F000053686F72745F4E756D5F323A256C750D04
:106F10000A000000556454656D706543685F4E75E6
:106F20006D5F323A256C750D0A000000556454659A
:106F30006D70654469735F4E756D5F323A256C758F
:106F40000D0A00004F7654656D706543685F4E759D
:106F50006D5F323A256C750D0A0000004F7654655E
:106F60006D70654469735F4E756D5F323A256C755F
:106F70000D0A0000440000206374725F74656D7038
:106F8000657261747572655B305D3A25640D0A0047
:106F90006374725F74656D70657261747572655B40
:106FA000315D3A25640D0A004261747465725F5662
:106FB0006F6C3A256C750D0A00000000040000207B
:106FC00063625F76616C5F6C6173743A25640D0A6D
:106FD000000000000500002063625F6F7065726151
:106FE00074655F73746174653A25640D0A0000006E
:106FF000C001002040070020424D535F313A256414
:107000000D0A0000424D535F323A25640D0A00001C
:10701000270000206D6F64653A25640D0A000000AA
:107020006D6F6465000000007465737400000000FB
:107030007465737420737563636573732100000056
:107040006A69616F7A68756E000000006A69616F35
:107050007A68756E20737563636573732100000031
:107060007065697A686900007065697A686920737B
:10707000756363657373210063657368690000005D
:1070800063657368692073756363657373210000BA
:107090007475696368750000747569636875207339
:1070A0007563636573732100636163687500000035
:1070B0006361636875207375636365737321000092
:1070C000C002002010B54FF480712648FEF794FAF4
:1070D000044624480078A04233D00C2222A1214843
:1070E000FBF757F830BB2448007818BB012002F0AA
:1070F0001DFF012080F3138800BF00BF00BF00BF49
:1071000000BF00BFBFF34F8F00BF00BF00BF1B48D1
:10711000006800F4E0601A490843001D1749086040
:1071200000BF00BF00BFBFF34F8F00BF00BF00BF55
:1071300000BFFEE722460B49222000F0FBFD0020A5
:1071400010BD0848007808280AD9064800F07AF8E7
:1071500030B922460349222000F0ECFD0020EFE781
:107160000120EDE7340600207A68656E676A69637E
:107170006573686900000000840000200CED00E0E9
:107180000000FA0510B54FF480712648FEF71AFA90
:10719000044624480078A04233D00C2222A1214882
:1071A000FAF7F7FF30BB2448007818BB012002F043
:1071B000BDFE012080F3138800BF00BF00BF00BFE9
:1071C00000BF00BFBFF34F8F00BF00BF00BF1B4811
:1071D000006800F4E0601A490843001D1749086080
:1071E00000BF00BF00BFBFF34F8F00BF00BF00BF95
:1071F00000BFFEE722460B49232000F09BFD002044
:1072000010BD0848007808280AD9064800F0EAF8B6
:1072100030B922460349232000F08CFD0020EFE71F
:107220000120EDE7D80700207A68656E676A696318
:107230006573686900000000840000200CED00E028
:107240000000FA052DE9F0410646374600BF787880
:107250005C490978884204D1B879162801D1F879B7
:1072600000B9ACE058480021016041608160574896
:10727000006820F0080055490860554C002084F84B
:10728000950001205349087000205349087020469A
:1072900090F8940018B103205049087002E00220D1
:1072A0004E490870BD880020B8803A783146381DB4
:1072B000FEF7D2F88046B8F1010F02D1B888A84293
:1072C00000D07CE00825711915222046FAF736FF18
:1072D0001535207D00F0010000B970E0207D000927
:1072E00010283AD2DFE800F008090A0B0C0D17212C
:1072F0002B3639353939373830E02FE02EE02DE0A4
:107300002CE07119262204F11500FAF717FF05F198
:10731000260085B222E071192A2204F13B00FAF717
:107320000DFF05F12A0085B218E071191F2204F142
:107330006500FAF703FF05F11F0085B20EE0711931
:1073400088200A68C4F8842009790155681D85B22F
:1073500004E003E002E001E000E000BF00BF94F8B9
:107360008C00217DB0EB111F26D104F1800000219B
:10737000C16001611A480078401C1949087008462C
:1073800000785A2805DD062084F88C00002008705B
:1073900012E0134800783C2803DD072084F88C00B5
:1073A0000AE00F4800781E2803DD082084F88C00CE
:1073B00002E0002084F88C000120BDE8F08100BFCD
:1073C0000020FAE72A0000203407002000000020F7
:1073D0004007002032000020300000203100002053
:1073E000370000202DE9F0410646374600BF787887
:1073F0005C490978884204D1B879162801D1F87916
:1074000000B9ACE0584800210160416081605748F4
:10741000006820F0100055490860554C002084F8A1
:1074200095000120534908700020534908702046F8
:1074300090F8940018B103205049087002E002202F
:107440004E490870BD880020B8803A783146381D12
:10745000FEF722F88046B8F1010F02D1B888A842A1
:1074600000D07CE00825711915222046FAF766FE47
:107470001535207D00F0010000B970E0207D000985
:1074800010283AD2DFE800F008090A0B0C0D17218A
:107490002B3639353939373830E02FE02EE02DE002
:1074A0002CE07119262204F11500FAF747FE05F1C8
:1074B000260085B222E071192A2204F13B00FAF776
:1074C0003DFE05F12A0085B218E071191F2204F172
:1074D0006500FAF733FE05F11F0085B20EE0711961
:1074E00088200A68C4F8842009790155681D85B28E
:1074F00004E003E002E001E000E000BF00BF94F818
:107500008C00217DB0EB111F26D104F180000021F9
:10751000C16001611A480078401C1949087008468A
:1075200000785A2805DD062084F88C0000200870B9
:1075300012E0134800783C2803DD072084F88C0013
:107540000AE00F4800781E2803DD082084F88C002C
:1075500002E0002084F88C000120BDE8F08100BF2B
:107560000020FAE738000020D808002000000020A2
:10757000E40800203B000020390000203A000020F1
:107580003F00002000BFFEE701480079704700007F
:10759000FC1000202DE9F0412748006800044FEA64
:1075A0009018A8F5406000F100642546202123488A
:1075B000FAF7DDFD288840F2253188420CD00846D4
:1075C0001E49088200221E491C48C0E906211021DC
:1075D000103001F0CDFB28E0184895E84E0010303F
:1075E0004EC01649D1E906610022164B3046FAF723
:1075F000DFFF08D2002213491048C0E906211021FC
:10760000103001F0B5FB0D49D1E9066100220E4BA7
:107610003046FAF7E5FF08D200220B490748C0E9D7
:1076200006211021103001F0A3FB0120074908704A
:1076300000204880BDE8F081E0F7FF1FA001002096
:1076400000C0824000C0724000E08540220000205F
:1076500070B55148007800287ED05048007850B965
:107660004F480078032800D170BD0320FCF768F96B
:1076700003280BD1F8E74A480078042800D1F3E743
:107680000420FCF75DF9042800D1EDE744480078B8
:1076900000287CD0012804D002283BD0042875D1D2
:1076A00076E04FF480513F4803F052FED8B13E4897
:1076B000C07C00F01000102803D10220FCF740F934
:1076C00027E03A480078012823D1FBF75BFC044609
:1076D000FBF744FC844202DA0220FCF731F9022075
:1076E0003249087015E030484468002C01DB204620
:1076F00000E06042B0F57A7F0BDCFBF743FC054607
:10770000FBF72CFC00F5FA70854202DD0220FCF745
:1077100017F93EE04FF48051224803F019FEE0B122
:107720002348C07C00F01000102803D10120FCF792
:1077300007F928E01D480078012824D1FBF70EFC4A
:107740000446FBF71FFC844202DA0120FCF7F8F83C
:1077500002201649087016E01CE015484468002C09
:1077600001DB204600E06042B0F57A7F0BDCFBF7DE
:10777000F5FB0546FBF706FC00F5FA70854202DDD5
:107780000120FCF7DDF804E001E0FFE700BF00BFE7
:1077900000BF00BF00BF67E70E0000200F00002001
:1077A00005000020000C0140400700201D000020C3
:1077B000E40800200148C078C0097047880900200B
:1077C00010B52A48B0F80D4024F0100424F020042D
:1077D00024F0800424F004044FF48051244803F082
:1077E000B7FD40B124F0020424F4006424F40054F2
:1077F00024F4004405E024F0010424F4804424F43B
:10780000805400BF1B484078012800D12BE01A4863
:10781000007800B127E019480078042809D1042134
:10782000174803F08DFD08B9012000E0002000B9E1
:1078300019E0FFF7BFFF00B115E001F043FA00B90E
:1078400011E02CB10948B0F80D000E4908800AE09B
:107850000D480078032800D005E00C48007800B1FE
:1078600001E0012010BD00BF0020FBE74007002021
:10787000000C0140180100201B0000200500002022
:1078800000100140340000203100002036000020AC
:1078900010B52A48B0F80D4024F0100424F020045C
:1078A00024F0800424F004044FF48051244803F0B1
:1078B0004FFD40B124F0020424F4006424F4005489
:1078C00024F4004405E024F0010424F4804424F46A
:1078D000805400BF1B484078022800D12BE01A4892
:1078E000007800B127E019480078042809D1022166
:1078F000174803F025FD08B9012000E0002000B979
:1079000019E0FFF757FF00B115E001F0E1F900B908
:1079100011E02CB10948B0F80D000E4908800AE0CA
:107920000D480078032800D005E00C48007800B12D
:1079300001E0012010BD00BF0020FBE7E4080020AB
:10794000000C0140180100201C0000200500002050
:10795000001001403C0000203A0000203E000020C2
:1079600010B540F2026004F059F94FF4C06004F021
:1079700055F940F2096004F051F9032003F0F2FFD9
:10798000202303220021024803F084FC10BD0000E4
:107990000008014000B501F071FD00BD10B502F016
:1079A0003FFB01200749087000204880064800215D
:1079B0000180002403E003F0BFFB601CC4B2022C72
:1079C000F9D310BD400000204400002038B500204D
:1079D0000090441E6946052002F089FD012800D070
:1079E0000BE0BDF8000040F6E44148436521484300
:1079F00040F6FF71B0FBF1F400BF204638BD10B572
:107A000002F030FB10BD00BFFEE710B5FDF7C2FC71
:107A100010BD000010B5002807DA0A07140E054A49
:107A200000F00F031B1FD45403E00A07130E024A91
:107A3000135410BD18ED00E000E400E02DE9F04122
:107A400005464FF096080B20244981F88C0035B18B
:107A5000012D02D0022D08D103E0032407E0002409
:107A600005E004244FF4FA6801E0002400BF00BFE1
:107A70001A48C0F890401A48006820F001001849E0
:107A8000086001F0E3FA6006040E002700261CE0FF
:107A90000A2003F0C7F81248007800F0010090B106
:107AA0000F48006820F001000D490860FFF70AFB4D
:107AB000022D06D00948C07C2040A04202D10127F7
:107AC00000E0012706E0701C86B20A2098FBF0F067
:107AD000B042DDDC00BF78B2BDE8F0814007002095
:107AE000000000202DE9F04105464FF096080B20DC
:107AF000244981F88C0035B1012D02D0022D08D126
:107B000003E0032407E0002405E004244FF4FA68AE
:107B100001E0002400BF00BF1A48C0F890401A4896
:107B2000006820F004001849086001F07DFB600641
:107B3000040E002700261CE00A2003F073F8124808
:107B4000007800F0040090B10F48006820F00400B5
:107B50000D490860FFF716FB022D06D00948C07CCE
:107B60002040A04202D1012700E0012706E0701C5E
:107B700086B20A2098FBF0F0B042DDDC00BF78B29C
:107B8000BDE8F081E40800200000002070470000FC
:107B900070B504460D4684B100224FF48051184858
:107BA00003F026FB01220821164803F021FB0020E8
:107BB0001549087000F066F91CE001220421114803
:107BC00003F016FB0020FAF765FE012211030C48B2
:107BD00003F00EFBFAF70EFF0121002000F01AF867
:107BE0000020FAF7F1FE00220821064803F000FB0E
:107BF00001F044FC054804700548057070BD0000A4
:107C000000080140000C01401E0000200D00002073
:107C10002600002070B504460D4600212046FDF7E1
:107C200013F822462021034803F0E2FA02480570C7
:107C300070BD0000000C0140ED00002010B51B4895
:107C400090F8940018B104201949087002E001204E
:107C500017490870154890F8950000B110BD15211E
:107C60001248FAF784FA262110481530FAF77FFAFD
:107C70002A210E483B30FAF77AFA1F210B4865306B
:107C8000FAF775FA09488030002141600172C1603D
:107C900001610120054981F89500052081F88C00DB
:107CA00000200449087000BFD8E70000400700200A
:107CB000310000203200002010B51B4890F89400DD
:107CC00018B104201949087002E001201749087012
:107CD000154890F8950000B110BD15211248FAF72B
:107CE00046FA262110481530FAF741FA2A210E48A3
:107CF0003B30FAF73CFA1F210B486530FAF737FAA8
:107D000009488030002141600172C1600161012099
:107D1000054981F89500052081F88C000020044970
:107D2000087000BFD8E70000E40800203A000020F7
:107D30003B000020704710B5012003F0E7FF10B1B1
:107D4000012003F0DBFF022003F0E0FF68B1022016
:107D500003F0D4FF4FF4003002F0DAFF03F0EAFF43
:107D6000002003F0BBFF03F0E5FF10BD10B50022BB
:107D70000121032003F0DAFC40F21B7003F04EFFF8
:107D800040F21C7003F04AFF03F030FD02F0A2FC49
:107D9000002211464FF4003002F056FF4FF400303D
:107DA00002F0B6FF4FF4003002F0AAFF4FF410606B
:107DB00003F0B4FE4FF4106003F0C0FE4FF4007007
:107DC00003F05CFF40F60F0003F028FF03F0CCFF48
:107DD00003F0B0FF022003F0A5FF03F0ABFF282063
:107DE00003F0B2FF03F0A6FF03F0A4FF4FF47A7094
:107DF00003F050FF03F09EFF10BD000010B51021EE
:107E0000014801F087F810BD2806002010B50321B5
:107E1000014801F07FF810BDCA03002010B5082109
:107E2000014801F077F810BDD404002010B50C21F2
:107E3000014801F06FF810BDDE05002010B5FDF718
:107E4000B9FB08B9012010BD094800680849496814
:107E5000884201D20120F6E70548807A28B104481B
:107E60004068322801D80120EDE70020EBE7000050
:107E7000A001002000B9704700210160018100BF0E
:107E8000F9E70000002002490870488070470000B0
:107E90008C00002010B54FF480710348FAF767F9A1
:107EA00000200249088010BDFA0F0020AE0000201B
:107EB00010B54FF480710348FAF759F900200249D0
:107EC000088010BD0C120020F20000202DE9F047C0
:107ED0008AB005466E68686800880890BDF8200082
:107EE00043F20D12811A904274D014DC43F2061250
:107EF000A0EB020190426ED008DCB0F5445F17D0D1
:107F0000A0F544500538002867D175E0012970D0EC
:107F10000629F9D188E003296CD004DC01296AD054
:107F20000229F1D105E1042970D07429ECD162E174
:107F3000E878C0F3C100012802D1CD48007818B11B
:107F400001200AB0BDE8F087022400222146641C0B
:107F5000725430191422C749FAF7F0F8C648007B6A
:107F6000B8B3C548C07AC3494978884203D1C248EA
:107F7000007BF07039E0FFF723FC68B3BD49487817
:107F8000FAF7D7FACDE90001BB49D1E906733A46C1
:107F90000199FAF7E4F90022B84BCDE90201FAF7AA
:107FA000DEF90022B64BCDE90401FAF74AFACDE931
:107FB0000601FAF7E4FA1FFA80FA0A209AFBF0F1B8
:107FC00000FB11A0052809DB0A209AFBF0F0401CF9
:107FD000F0700AE059E03EE005E00EE10A209AFB6D
:107FE000F0F0F07001E00020F07004F1140084B2B1
:107FF00005E184E0BFE063E0E878C0F3C100012858
:1080000002D19B48007810B101209AE7D7E0022402
:1080100000222146641C72543019122295491531F0
:10802000FAF78CF81234EAE0E878C0F3C1000128CE
:1080300002D18F48007808B1012082E70224002293
:108040002146641C7254301914228A492731FAF7E8
:1080500075F81434D3E0E878C0F3C100012802D1E8
:108060008348007808B101206BE7022400222146F2
:10807000641C7254DFF8FC9109F13B0930190E229F
:108080004946FAF75BF80E34B9E0E878C0F3C1006E
:10809000012802D17648007808B1012051E7022476
:1080A00000222146641C7254DFF8C89109F13B0993
:1080B0003019102209F10E01FAF740F810349EE051
:1080C000E878C0F3C100012802D16948007808B1FE
:1080D000012036E7022400222146641C7254DFF896
:1080E000949109F13B093019D9F81E100160D9F8B3
:1080F00022104160D9F8261081600C347FE0E878C6
:10810000C0F3C100012802D15948007808B101200C
:1081100017E7022400222146641C7254DFF85491B0
:1081200009F1650930190D224946FAF707F80D34AF
:1081300065E0E878C0F3C100012802D14C4800781E
:1081400008B10120FDE6022400222146641C72547D
:108150002146641C7254DFF81C9109F1650930193D
:10816000D9F80D100160D9F811104160D9F8151037
:1081700081600C3443E0E878C0F3C100012802D1EB
:108180003B48007808B10120DBE6022400222146AA
:10819000641C72542146641C7254DFF8D89009F1B3
:1081A00065093019D9F819100160B9F81D108180DE
:1081B000A41D3019002101608180A41D1FE0E87812
:1081C000C0F3C100012802D12948007808B101207C
:1081D000B7E6022400222146641C7254DFF8949012
:1081E00009F184093019D9F80010016099F80410D8
:1081F0000171641D03E00020A3E60020A1E600BF9A
:10820000E87820F018001030E870B5F80100810817
:10821000288861F3C9002880B5F8010020F4FE70B9
:1082200000F58470A5F80100A87820F03E00801CBD
:10823000A870601EC11700EB5171C9104A1C6988F3
:1082400062F38A116980E87820F0E000E8702C8100
:108250000221284600F05EFE38B90A48006840F462
:1082600080700849086000206BE6012069E6000084
:108270006E00002040070020A001002000002440E4
:1082800000408F40000000202DE9F04788B00546EF
:108290006E68686800880690BDF8180043F20D22E9
:1082A000811A904273D014DC43F20622A0EB020143
:1082B00090426DD008DCB0F5485F17D0A0F548506B
:1082C0000538002876D16BE0012974D00629F9D150
:1082D00082E0032970D004DC01296ED00229F1D19B
:1082E000FFE004296AD07429ECD15CE1E878C0F39E
:1082F000C100012802D1CA48007818B1012008B095
:10830000BDE8F087022400222146641C7254301913
:108310001422C449F9F712FFC348007B88B3C2484E
:10832000C07AC0494978884203D1BF48007BF070C9
:1083300032E0FFF7ADFA60B3BA494878FAF7F9F8D6
:10834000CDE90001B849D1E906733A460199FAF737
:1083500006F80022B54BCDE90201FAF772F8CDE933
:108360000401FAF70CF900F0FF0A0A209AFBF0F179
:1083700000FB11A0052805DB0A209AFBF0F0401C49
:10838000F07009E00A209AFBF0F0F07004E054E08D
:1083900039E0FFE70020F07004F1140084B206E138
:1083A000E878C0F3C100012802D19D48007830B1BF
:1083B0000120A4E7F9E07AE0B5E059E0D7E0022433
:1083C00000222146641C725430191222954915313D
:1083D000F9F7B4FE1234EAE0E878C0F3C1000128EE
:1083E00002D18F48007808B1012088E702240022DA
:1083F0002146641C7254301914228A492731F9F736
:108400009DFE1434D3E0E878C0F3C100012802D106
:108410008348007808B1012071E702240022214638
:10842000641C7254DFF8FC9109F13B0930190E22EB
:108430004946F9F783FE0E34B9E0E878C0F3C1008D
:10844000012802D17648007808B1012057E70224BC
:1084500000222146641C7254DFF8C89109F13B09DF
:108460003019102209F10E01F9F768FE10349EE070
:10847000E878C0F3C100012802D16948007808B14A
:1084800001203CE7022400222146641C7254DFF8DC
:10849000949109F13B093019D9F81E100160D9F8FF
:1084A00022104160D9F8261081600C347FE0E87812
:1084B000C0F3C100012802D15948007808B1012059
:1084C0001DE7022400222146641C7254DFF85491F7
:1084D00009F1650930190D224946F9F72FFE0D34CF
:1084E00065E0E878C0F3C100012802D14C4800786B
:1084F00008B1012003E7022400222146641C7254C3
:108500002146641C7254DFF81C9109F16509301989
:10851000D9F80D100160D9F811104160D9F8151083
:1085200081600C3443E0E878C0F3C100012802D137
:108530003B48007808B10120E1E6022400222146F0
:10854000641C72542146641C7254DFF8D89009F1FF
:1085500065093019D9F819100160B9F81D1081802A
:10856000A41D3019002101608180A41D1FE0E8785E
:10857000C0F3C100012802D12948007808B10120C8
:10858000BDE6022400222146641C7254DFF8949058
:1085900009F184093019D9F80010016099F8041024
:1085A0000171641D03E00020A9E60020A7E600BFDA
:1085B000E87820F018001030E870B5F80100810864
:1085C000288861F3C9002880B5F8010020F4FE7006
:1085D00000F58470A5F80100A87820F03E00801C0A
:1085E000A870601EC11700EB5171C910491C6A8840
:1085F00061F38A126A80E87820F0E000E8702C814C
:108600000721284600F086FC38B90948006840F484
:10861000007007490860002071E601206FE6000045
:1086200080000020E4080020A001002000408F40CE
:10863000000000202DE9F843064675680027B8467B
:10864000706800880090BDF80000B0F5854F6ED0CE
:108650000BDCA0F584400C286AD2DFE800F0325E23
:10866000A1B1C1D7F3F1F0EFEEED44F20532811A7A
:1086700090427DD016DC44F20132A0EB0201904220
:1086800077D00ADCA0F58440A0F1F500002871D075
:10869000012870D003284BD1A5E201296CD0022912
:1086A000F9D1D4E1032968D004DC012966D002297C
:1086B000F1D148E2132972D0A1F2FB410029EAD19D
:1086C0007AE2F078C0F3C100012802D1F8480078BE
:1086D00010B10120BDE8F8834FF48440F5490880CB
:1086E000002088700C2422462846F9F727FDF2481E
:1086F00002782146641C6A54F04802782146641CC2
:108700006A54EF4802782146641C6A540088C0F31A
:1087100007222146641C6A546CE2F078C0F3C10061
:10872000012802D1E248007818B10120D2E753E2D3
:108730005EE20224E348007848B100222046611C32
:108740008CB22A542046611C8CB22A5426E0285D43
:10875000002818DD285D052815DA285DDA49097832
:10876000884202D0285DFBF7EBF80022204606E0A5
:108770007DE123E132E232E252E1F4E1BAE1611C4F
:108780008CB22A5404E001222046611C8CB22A5487
:10879000CD4802782046611C8CB22A542AE276E148
:1087A000F078C0F3C100012802D1C148007808B1B7
:1087B00001208FE7022400222146641C6A5419E23A
:1087C000F078C0F3C100012802D1B948007808B19F
:1087D00001207FE7022400222146641C6A5409E23A
:1087E000F078C0F3C100012802D1B148007808B187
:1087F00001206FE7022400222146641C6A542819D4
:108800001422B249F9F79AFC1434F3E1F078C0F37A
:10881000C100012802D1A648007808B1012059E71B
:10882000022400222146641C6A5428191222A849F5
:10883000F9F784FC1234DDE1B7E0A5E09AE03DE011
:1088400010E0FFE7F078C0F3C100012802D198489A
:10885000007808B101203DE7022400222146641C73
:108860006A54C7E14FF00008AC78012C01D0022C0B
:108870001CD1012C04D1012001F018FAC7B203E089
:10888000012001F061FAC7B26FB10120914908706F
:10889000A878487028794880E878897840EA0120EB
:1088A0008C49488004E04FF0030801E04FF00108D4
:1088B00002242146641C05F801809BE14FF000086A
:1088C000EC78A87840EA042482484088A04249DB3A
:1088D00080488088A04204D07E488088401CA04206
:1088E0003DD16C79287940EA0424802C34D80220C8
:1088F00078490870E8788880A878097940EA0120EA
:10890000744988806879C8802879897940EA01208B
:108910007049C8800846C288A91D0830F9F70EFCC6
:108920006C484078012804D1022001F0BFF9C7B299
:1089300003E0022001F008FAC7B257B16548808809
:108940006449498888420FD188216248F9F70FFCB1
:108950000AE04FF0040807E04FF0030804E04FF08E
:10896000020801E04FF0010802242146641C05F8CA
:1089700001803FE188215748F9F7F9FB02240022E2
:108980002146641C6A5435E1F078C0F3C100012827
:1089900002D14748007808B101209BE602244E48E6
:1089A000027B2146641C6A5424E1012001F0BEFAD6
:1089B000022400222146641C6A541BE1F078C0F3B3
:1089C000C100012802D13A48007808B1012081E6AF
:1089D000022400222146641C6A5440480078012881
:1089E00018D140213E4802F0ABFC08B9012200E05A
:1089F00000222046611C8CB22A54642039494880E8
:108A00000120394908700020488038494880384999
:108A1000086004E000222046611C8CB22A54E9E080
:108A2000F078C0F3C100012802D12148007808B1D4
:108A300001204FE6022400222146641C6A541021C2
:108A4000274802F085FC2246641CA854D2E0F07846
:108A5000C0F3C100012802D11548007808B10120F7
:108A600038E6022400222146641C6A54C2E0F078F1
:108A7000C0F3C100012802D10D48007808B10120DF
:108A800028E6022400222146641C6A54B2E0F078F1
:108A9000C0F3C100012802D10548007808B10120C7
:108AA00018E6022400222146641C6A54A2E0000059
:108AB0004800002094090020ED000020260000203E
:108AC000940000200E00002005000020002A00086D
:108AD0000401002018010020A00100200D0000204A
:108AE000000C0140C4000020DC000020C800002071
:108AF000E8000020F078C0F3C100012802D15948F5
:108B0000007808B10120E5E5022400222146641C1A
:108B10006A545548007801280FD10121534802F0CA
:108B20000FFC08B9012200E000222046611C8CB233
:108B30002A5464204E49488004E000222046611CEB
:108B40008CB22A5456E0F078C0F3C100012802D15B
:108B50004448007808B10120BCE5022400222146E7
:108B6000641C6A5446E0F078C0F3C100012802D1C9
:108B70003C48007808B10120ACE5022400222146DF
:108B8000641C6A543848007801280FD10121374805
:108B900002F0D6FB08B9012200E000222046611C49
:108BA0008CB22A5464203249488004E000222046D6
:108BB000611C8CB22A541DE0F078C0F3C10001287A
:108BC00002D12848007808B1012083E50224002260
:108BD0002146641C6A540DE000207BE500BF03249D
:108BE0000020A87006E0284602F032FE044601E0AC
:108BF00000206FE500BFF07820F018001030F07012
:108C0000B6F801008108308861F3C9003080B6F8F9
:108C1000010020F4FE7000F58470A6F80100B07821
:108C200020F03E00801CB070601EC11700EB517137
:108C3000C910491C728861F38A127280F07820F0A2
:108C4000E000F07034810B21304600F063F938B950
:108C50000848006840F4806006490860002039E553
:108C6000012037E5480000200D00002000140140DD
:108C7000CC0000200000002010B5044622464FF42E
:108C80000051064802F0B4FA0CB9012000E00020BF
:108C900002460421014802F0ABFA10BD000C01406D
:108CA00007480078022806D005480078032802D03B
:108CB0000348007808B9012070470020FCE7000055
:108CC00005000020014800787047000032000020B5
:108CD00001480078704700003B000020704700000A
:108CE00070B504460D46214801F08AFB002001F0D2
:108CF0004DFC012211021D4801F0BFFC00211B4860
:108D000001F072FB01221146184801F04AFB0523CD
:108D100022460021154801F047FC4FF46022012152
:108D2000124801F0C1FB01221146104801F09DFBE1
:108D30000E4801F091FB012001F074FF0B4801F097
:108D40001BFB0121094801F089FC00BF02210748F3
:108D500001F0C6FB0128F9D1044801F07BFC288012
:108D60000221024801F0B8FB012070BD002401403F
:108D70002DE9F04705460E461548006800044FEA05
:108D80009018A8F5406000F10067002440F22539F2
:108D900002F026F9FCF7F8FA384602F0ABF8FCF7D7
:108DA000F3FA02F091F802F01BF900BF0AE028196B
:108DB000D0F800903819494602F034F9FCF7E4FA8B
:108DC000201DC4B2B442F2DB02F07EF8BDE8F087A9
:108DD000E0F7FF1F10B510210148FFF7C9FF10BDD4
:108DE000B00100200A48007888B109484088401C3A
:108DF0000749488008464088B0F5167F07DD002007
:108E000048800448006840F4000002490860704748
:108E1000220000200000002010B50024FEF7D0FC46
:108E2000C0B1FEF735FD98B10D4880680D498968DD
:108E3000884206D3FEF7A8FB08B102240EE0012405
:108E40000CE0FEF7A1FB08B1012407E0022405E0D5
:108E5000012403E0FEF71CFD00B10224204610BDF2
:108E600040070020E408002010B50024FEF7A8FC0D
:108E7000C0B1FEF70DFD98B11248806812498968AB
:108E8000884206D3FEF780FB08B1022418E00124D3
:108E900016E0FEF779FB08B1012411E002240FE08F
:108EA00001240DE0FEF7F4FC08B1022408E00548B7
:108EB000806805498968884201D2022400E00124C3
:108EC000204610BD40070020E408002070B505468C
:108ED0000C461DB114B1B4F5807F01D9002070BDDE
:108EE000224629460748F9F729F900200649088053
:108EF0000648046040F20631054803F024FB0120D7
:108F0000EDE700000C110020F0000020F40000202C
:108F10000044004070B586B004460E4600252CB1D2
:108F20002648007810B92648007810B9002006B00D
:108F300070BD2448216801602089224908810B46C0
:108F40001A8961685868F9F7F9F8142101A8F9F746
:108F50000EF91C480568E808029004208DF80C0002
:108F600000208DF80D0017480089082803DD08202F
:108F70008DF80E0003E01348007A8DF80E009DF87E
:108F80000E20104841680DF10F00F9F7D7F801A93C
:108F90000D4801F04FFD032801D10020C7E7094823
:108FA0004088C0F38410012806D0012003490870CE
:108FB0000121054801F0C7FC0120B8E7A800002006
:108FC0000D000020F00E00200064004070B5054642
:108FD0000C461DB114B1B4F5807F01D9002070BDDD
:108FE000224629460948F9F7A9F8002008490880CF
:108FF0000848046040F20631074803F0A4FA40F242
:109000000631054803F0ACFA0120E8E7FA0E00202B
:10901000AC000020B00000200038014010B504482A
:10902000007800B110BD00F011F800BFFAE70000B1
:109030003000002010B50448007800B110BD00F0E9
:10904000F3F800BFFAE70000390000202DE9F041F5
:109050006E4C25466E4E082020706E480078607079
:109060004220A0701020E0701620A0710020A08087
:10907000E07100212278501C2070A9542278501CE5
:109080002070A9542278501C2070A9542278501CBA
:109090002070A9542278501C2070A9542278501CAA
:1090A0002070A95496F88C102278501C2070A95476
:1090B000594801782278501C2070A9540021227848
:1090C000501C2070A9542278501C2070A95422787A
:1090D000501C2070A9542278501C2070A95422786A
:1090E000501C2070A9542278501C2070A95422785A
:1090F000501C2070A95496F88C0010286AD2DFE822
:1091000000F008090A5A5B5C5D5E6968695F69691D
:10911000666760E05FE090208059032802D0042851
:1091200047D106E09020815D2278501C2070A95420
:109130003FE09020815D2278501C2070A954374870
:1091400081782278501C2070A9543448408801123C
:109150002278501C2070A95400212278501C2070C5
:10916000A9542278501C2070A9542C4801792278E7
:10917000501C2070A9542948808801122278501C64
:109180002070A95400212278501C2070A954227804
:10919000501C2070A9542149CA88217848191F49B8
:1091A0000831F8F7CBFF20781C49897908442070F2
:1091B00000BF00BF0FE00EE00DE00CE00BE00AE0A6
:1091C0009020815D2278501C2070A95403E002E0B9
:1091D00001E000E000BF00BF22782146201DFCF71F
:1091E0003BF90746012F02D00020BDE8F08121782D
:1091F0002846FFF7EBFE012009490870002048804F
:1092000001200849087000BFEFE700003406002085
:10921000400700202A000020330000201801002011
:1092200034070020300000202DE9F0416E4C254627
:109230006E4E082020706E48007860704220A0704A
:109240001020E0701620A0710020A080E0710021A5
:109250002278501C2070A9542278501C2070A954E8
:109260002278501C2070A9542278501C2070A954D8
:109270002278501C2070A9542278501C2070A954C8
:1092800096F88C102278501C2070A9545948017807
:109290002278501C2070A95400212278501C207084
:1092A000A9542278501C2070A9542278501C207098
:1092B000A9542278501C2070A9542278501C207088
:1092C000A9542278501C2070A9542278501C207078
:1092D000A95496F88C0010286AD2DFE800F008093B
:1092E0000A5A5B5C5D5E6968695F6969666760E030
:1092F0005FE090208059032802D0042847D106E07F
:109300009020815D2278501C2070A9543FE090206D
:10931000815D2278501C2070A954374881782278CA
:10932000501C2070A9543448408801122278501CE7
:109330002070A95400212278501C2070A954227852
:10934000501C2070A9542C4801792278501C2070A0
:10935000A9542948808801122278501C2070A954F1
:1093600000212278501C2070A9542278501C2070B3
:10937000A9542149CA88217848191F490831F8F7AA
:10938000DDFE20781C4989790844207000BF00BFA9
:109390000FE00EE00DE00CE00BE00AE09020815DB4
:1093A0002278501C2070A95403E002E001E000E0A4
:1093B00000BF00BF22782146201DFCF76DF807464C
:1093C000012F02D00020BDE8F08121782846FFF768
:1093D0007DFD0120094908700020488001200849CE
:1093E000087000BFEFE70000D8070020E408002065
:1093F000380000203300002018010020D808002089
:10940000390000201048007820B10F484088401CE7
:109410000D4948800D480078A0B10C484088401C98
:109420000A4948800846408841F28831884203DC76
:1094300001200749087005E0044800210160002070
:109440000349087070470000120000201600002039
:109450001A0000200649097849B90649087118B16F
:109460000221054A117002E00321034A117070477E
:10947000EC000020FC1000203300002001200249F5
:1094800008700020488070478C0000200748007852
:1094900058B106484088401C80B204494880B0F565
:1094A000C87F02DB0846002101607047DC00002015
:1094B00070B5024600231AE0002012E032F8106076
:1094C000451C32F81550AE4209DD32F81040451CFB
:1094D00032F8155022F81050451C22F81540451C52
:1094E000A8B2CD1A6D1E8542E8DC5D1CABB24D1EE4
:1094F0009D42E1DC70BD000001480078704700002B
:109500003100002010B500F067FC0948002101601F
:109510004160816098210748F8F729FE012006493B
:109520000870002048800520024981F88C0010BD99
:1095300034070020400700202C0000200748007856
:10954000052809D2DFE800F003040506070003E060
:1095500002E001E000E000BF00BF704731000020E2
:1095600001480078704700003A00002010B500F074
:1095700089FC07480021016041608160982105480D
:10958000F8F7F5FD0520034981F88C0010BD0000B7
:10959000D8080020E408002007480078052809D2F0
:1095A000DFE800F003040506070003E002E001E045
:1095B00000E000BF00BF70473A00002010B5B1487E
:1095C0000088401C80B2AF490880B0F57A7F1EDB6E
:1095D000AD480068401CAC4908600020A9490880DB
:1095E00000BFAA48007878B1A8484088401C80B2E3
:1095F000A6494880012807DB00204880A44800686D
:1096000040F02000A249086000BFFFF7EBFBA14833
:10961000006820B19F480068401E9E490860F9F725
:109620007BF900BF9C48007890B19B48408828B1E6
:1096300099484088401E9849488009E0944800684D
:1096400040F001009249086000209349087048806A
:1096500000BF00BF9148007890B19048408828B181
:109660008E484088401E8D49488009E0884800683F
:1096700040F004008649086000208849087048804E
:1096800000BFF9F7E1F88648007818B384484088AD
:10969000401C80B28249488096281BDB002081490B
:1096A00008707F49087048800846007918B9012081
:1096B000087188600EE07A488068401C78498860AC
:1096C000032807D3002088607148006840F0080034
:1096D0006F4908607448007818B373484088401C8C
:1096E00080B27149488096281BDB00206F490870C2
:1096F0006D49087048800846007918B90120087142
:1097000088600EE068488068401C674988600328CC
:1097100007D3002088605E48006840F010005C4974
:1097200008606348007820B361484088401C604965
:10973000488008464088B0F5C87F0CDB0020488090
:109740005C484078022814D05148006840F08000FE
:109750004F4908600DE056484088C82809D155484F
:109760004078012805D04A48006840F04000484948
:1097700008605148007820B14F484088401C4E494D
:1097800048804E48407820B14C484088401C4B49A6
:1097900048804B48007820B149484088401C4849DF
:1097A00048804848007820B146484088401C4549D8
:1097B00048804548007820B143484088401C4249D1
:1097C00048804248007820B140484088401C3F49CA
:1097D00048803F48007820B13D484088401C3C49C3
:1097E00048803C480078D8B13A484088401C394904
:1097F000488008464088B0F5617F08DB012240219F
:10980000354801F0F5FC00203249488008E0314835
:109810004088C82804DB002240212F4801F0E8FCE2
:109820002E480078D8B12D484088401C2B494880EC
:1098300008464088B0F5617F08DB01228021264878
:1098400001F0D6FC00202549488008E023484088E4
:10985000C82804DB002280211F4801F0C9FCFAF768
:10986000A3F8FAF7D7F8FBF7E7FCF9F70DFBFFF7DA
:109870000DFEFBF7B7F8FFF7C5FDFBF769FDFCF739
:1098800027F810BD98000020940000204000002020
:109890000000002090000020B4000020F80000200C
:1098A0003407002030000020D808002039000020B4
:1098B0002C00002018010020B8000020E400002047
:1098C000BC000020C0000020C4000020C800002010
:1098D000CC000020D400002000100140D80000205F
:1098E00010B51448006840F00100124908600846AD
:1098F0004068114908400F494860084600680F4910
:1099000008400C4908600846006820F48020086080
:10991000084640680A490840064948600846006809
:1099200006490840034908604FF41F00886002F0B0
:1099300081FA10BD001002400C00FFE8FFFFF6FEA8
:10994000FFFF00F710B50121094802F019FD0128B9
:109950000CD10121064802F00FFD4FF0804002F0CB
:1099600089FC034802F086FCF9F7D0F910BD00002D
:109970000004004010B511210148FFF7CBFA10BDDB
:109980002806002010B504210148FFF7C3FA10BDD6
:10999000CA03002010B509210148FFF7BBFA10BD2A
:1099A000D404002010B50D210148FFF7B3FA10BD13
:1099B000DE05002010B505211E4802F098FD0128A3
:1099C00018D11C4802F03CFDC4B21B480088FF2897
:1099D00000D910BD00210846FBF708FC1648018895
:1099E0000088401C144A108014484454052101206A
:1099F000FBF7FCFB06210F4802F079FD012816D188
:109A00000F4800880F490968884205D340F20631A3
:109A1000084802F08BFDDCE7094802880088401CFA
:109A2000074B18800848815C024802F00EFD00BF19
:109A3000CFE7000000380140AE000020FA0F002000
:109A4000AC000020B0000020FA0E002010B5052167
:109A50001E4802F04CFD012818D11C4802F0F0FC11
:109A6000C4B21B480088FF2800D910BD0021084659
:109A7000FBF7CAFB164801880088401C144A108076
:109A80001448445405210120FBF7BEFB06210F4872
:109A900002F02DFD012816D10F4800880F490968F2
:109AA000884205D340F20631084802F03FFDDCE76A
:109AB000094802880088401C074B18800848815CD0
:109AC000024802F0C2FC00BFCFE7000000440040A3
:109AD000F20000200C120020F0000020F400002012
:109AE0000C11002010B586B000242D488078C0F3FA
:109AF00044002B494988C1F38411884246D0284844
:109B000080784008401C2649897860F34501244844
:109B10008170142101A8F8F72AFB21480468E008A5
:109B2000029004208DF80C0000208DF80D001C48D8
:109B30008078C0F3440020B119488078C0F3440015
:109B400000E02020441EE40015488078C0F3440063
:109B500013494988C1F38411884203D008208DF845
:109B60000E0005E00E48007A001BC0B28DF80E0012
:109B70009DF80E200A48406801190DF10F00F8F712
:109B8000DDFA01A9074800F055FF06E0002006496C
:109B900008700121034800F0D2FE06B010BD00009D
:109BA000F00E002000640040A800002070B586B0D0
:109BB00001AA0021394800F0CAFE9DF8170020B123
:109BC000012806D002280CD107E0354C4FF48076EE
:109BD00009E0344C4FF4807605E0334C4FF4807646
:109BE00001E006B070BD00BF9DF80C00029940EA8C
:109BF000C1009DF80D1040EA01052560A078C0F372
:109C0000440018B1A078C0F3440000E0202061882F
:109C1000C1F3841119B16188C1F3841100E02021DE
:109C2000884200DDDDE76088C0F3841018B16088E9
:109C3000C0F3841000E02020C500B54200D9D0E771
:109C4000A078C0F3440018B1A078C0F3440000E04D
:109C50002020451E616801EBC5009DF80E200DF126
:109C60000F01F8F76BFAA078C0F3440018B1A078A0
:109C7000C0F3440000E020206188C1F3841119B1D1
:109C80006188C1F3841100E02021884204D19DF84D
:109C90000E0000EBC500208100BFA2E70064004079
:109CA000D20E0020DC0E0020E60E00202DE9F0414F
:109CB000054640F2DC5725B1012D05D0022D15D106
:109CC0000BE00020BDE8F08102201D4981F88C00E6
:109CD00003211B48C0F890100AE00220184981F8BF
:109CE0008C0004211648C0F8901001E00020E9E73C
:109CF00000BF1448006820F0010012490860FFF717
:109D0000A5F90026002413E00A2000F08BFF0D487F
:109D1000007800F0010048B10A48006820F0010016
:109D200008490860FDF7CEF9C6B206E0601C84B2AF
:109D30000A2097FBF0F0A042E6DC00BF70B2C1E75A
:109D400040070020000000202DE9F041054640F2C8
:109D5000DC5725B1012D05D0022D0DD107E00020E3
:109D6000BDE8F0810E20194981F88C0006E00F2033
:109D7000164981F88C0001E00020F1E700BF14488B
:109D8000006820F0040012490860FFF74DFA002631
:109D9000002413E00A2000F045FF0D48007800F091
:109DA000040048B10A48006820F00400084908602F
:109DB000FDF7E8F9C6B206E0601C84B20A2097FB02
:109DC000F0F0A042E6DC00BF70B2C9E7E408002072
:109DD0000000002000BFFEE710B540F2026001F075
:109DE0001DFF4FF4C06001F019FF40F20E6001F05A
:109DF00015FF4FF4007303221821204801F04AFA9E
:109E00004FF48063032204211C4801F043FA1C48EC
:109E100002F020FB4FF41641194802F0C9FA002164
:109E2000174802F0D9FB0021154802F0C5FB0021BC
:109E3000134802F0B1FB0021114802F06FFB002132
:109E40000F4802F063FB04210D4802F0ADFB08212E
:109E50000B4802F0B9FB4FF4407001F0BDFC00224A
:109E60000121252001F062FC40F20531044802F096
:109E70006AFB034802F036FB10BD000000080140F9
:109E80000038014010B540F2026001F0C7FE4FF407
:109E9000C06001F0C3FE042303221821214801F011
:109EA000F9F90823032204211E4801F0F3F940F2D6
:109EB000117001F0B3FE1C4802F0CCFA4FF41641C9
:109EC000194802F075FA0021174802F085FB0021BD
:109ED000154802F071FB0021134802F05DFB0021E0
:109EE000114802F01BFB00210F4802F00FFB042178
:109EF0000D4802F059FB08210B4802F065FB4FF4B6
:109F0000407001F069FC00220121262001F00EFCC6
:109F100040F20531044802F016FB034802F0E2FA71
:109F200010BD000000080140004400402DE9F04150
:109F300005461348006800048609A6F5805000F124
:109F400000673DB142F2233401200E490870002021
:109F5000488001E04FF6FF7401F042F8FBF766FB22
:109F6000384600F0C7FFFBF761FB2146384600F09A
:109F70004BFFFBF75BFB00F0A7FFBDE8F0810000A3
:109F8000E0F7FF1F880000202DE9F04105461A4840
:109F9000006800044FEA9018A8F5006000F1006620
:109FA00000244FF6FF7701F01BF8FBF7EDF9304680
:109FB00000F0A0FF00BF0FE0FBF7E6F9601C2F5C8C
:109FC0004FF6FF7000EA0727285D0743301939462E
:109FD00000F01AFFA01CC4B2122CEDDB00F074FFDD
:109FE000A8F5006000F10066122231460348F8F738
:109FF000A5F8BDE8F0810000E0F7FF1F0401002094
:10A0000010B540F2036001F009FE4FF460430322F3
:10A010001021024801F03EF910BD0000000C014083
:10A0200010B540F2046001F0F9FD0823032210216D
:10A030000A4801F02FF940F2026001F0EFFD40F212
:10A04000096001F0EBFD032001F08CFC03231A46AC
:10A050000021034801F01EF910BD0000001001406E
:10A060000008014010B5202303220021014801F01F
:10A0700011F910BD000801400FB4054B10B503A93C
:10A08000044A029800F018F810BC5DF814FB0000B8
:10A09000E5B000080001002002E008C8121F08C156
:10A0A000002AFAD170477047002001E001C1121F59
:10A0B000002AFBD1704700002DE9FF4F8DB09B4671
:10A0C0000F460446002606E025280BD05A460F9975
:10A0D0009047641C761C20780028F5D111B03046DA
:10A0E000BDE8F08F0025A8460122984900E005430D
:10A0F00014F8013F203B02FA03F00842F7D1207820
:10A100002E2817D114F8010F45F004052A280ED087
:10A110006FF02F022078A0F1300109290AD808EB4E
:10A12000880102EB410100EB0108641CF2E757F8DB
:10A13000048B641C20786C280DD004DC4C2812D0D1
:10A140006A2811D104E074280DD07A280CD10AE0D5
:10A1500045F4001507E0617845F48015814202D18D
:10A16000641C05F58015641C2278692A45D008DC3A
:10A17000002AB3D0582A69D0632A10D0642A08D1A3
:10A180003BE0702A67D0732A13D0752A5CD0782AF6
:10A190005CD010465A460F999047761CD3E017F8CA
:10A1A000040B8DF8000000208DF80100E946012025
:10A1B00003E057F8049B4FF0FF3069074FF00005AC
:10A1C00001D40AE06D1C45450DDA8542FADB19F829
:10A1D00005100029F6D106E06D1C8542FCDB19F85C
:10A1E00005100029F8D12E4404E019F8010B5A4655
:10A1F0000F9990476D1EF8D2A5E00A200021CDE905
:10A200000801C5F3025002280DD001CFC117031E6B
:10A2100071F100030DDA4FF0000CD0EB0C006CEB89
:10A2200001012D2308E0FF1D27F00707F7E80201D1
:10A23000EDE72B0504D52B238DF8283001233BE0D7
:10A24000EB0739D02023F7E70A2000E01020002197
:10A25000CDE9080107E01020002145F00405CDE913
:10A2600008014FF00808C5F3025002280FD001CFB3
:10A2700000214FF0000A2B071FD5702A0DD0DDE911
:10A2800008C38CF0100C5CEA030C0CD015E0FF1D29
:10A2900027F00707F7E80201EBE740228DF82820B6
:10A2A0004FF0010A0BE050EA010306D030238DF88D
:10A2B00028308DF8292002239A46582A04D024A257
:10A2C0000DF120090B9209E026A2F9E7DDE9082348
:10A2D000F8F79EF90B9B9B5C09F8013D50EA0102DF
:10A2E000F4D1ADEB090020300890680701D44FF09D
:10A2F00001080899884502DDA8EB010000E0002074
:10A300008046002506E00AA85A46405D0F9990470E
:10A310006D1C761C5545F6DB04E030205A460F993B
:10A320009047761CB8F10001A8F10108F5DC05E0C2
:10A3300019F8010B5A460F999047761C0899481E48
:10A3400008900029F4DC641CC5E60000092801001F
:10A35000303132333435363738396162636465669B
:10A36000000000003031323334353637383941425D
:10A370004344454600000000816841F008018160C7
:10A3800000BF816801F008010029FAD1816841F01D
:10A390000401816000BF816801F004010029FAD145
:10A3A000704730B5012902D002291AD10CE0C36AE6
:10A3B00023F47003C362C36A541E4FF4700505EAA8
:10A3C00004542343C3620DE0836B23F4401383637F
:10A3D000836B541E4FF4401505EA045423438363F2
:10A3E00000E000BF00BF30BD21B1826842F40062CE
:10A3F000826003E0826822F400628260704700009D
:10A4000010B504461348204430B1B0F5806F0CD02D
:10A41000B0F5C05F1BD111E040F2093001F01EFC25
:10A4200040F2093001F00AFC12E040F20A3001F07B
:10A4300015FC40F20A3001F001FC09E040F20F3057
:10A4400001F00CFC40F20F3001F0F8FB00E000BF1F
:10A4500000BF10BD00DCFEBF816801F0010119B929
:10A46000816841F001018160704772B101F0010320
:10A470001BB1836843F48013836001F0020393B13E
:10A48000836843F4004383600DE001F001031BB1D6
:10A49000836823F48013836001F002031BB1836897
:10A4A00023F4004383607047012902D0022910D1B0
:10A4B00007E0836823F46023836083681343836029
:10A4C00008E0836823F4E043836083681343836078
:10A4D00000E000BF00BF704702688A430260704717
:10A4E0000246002013680B4003B1012070472DE99C
:10A4F000FE4F82460D461DB96FF00100BDE8FE8F8C
:10A5000000240EE0684600EB44015046FEF7E8FBED
:10A510008146B9F1000F02DC6FF00200EEE7601C2B
:10A52000C4B2062CEED30026002701240FE03DF82C
:10A5300016003DF81410884200DD26463DF817004D
:10A540003DF81410884200DA2746601CC4B2062C7D
:10A55000EDD3BE4204D1BDF8000028800120CDE734
:10A560004FF0000800240BE0B44207D0BC4205D0F5
:10A570003DF8140008EBA0001FFA80F8601CC4B27C
:10A58000062CF1D3A5F800800120B7E7054909683A
:10A5900021F47021034A11601146096801431160DA
:10A5A0007047000004240140F0B51D4606290CDA6E
:10A5B000436B01EB81071F26BE40B34301EB8106CD
:10A5C00002FA06F63343436322E00C290EDA036BEA
:10A5D0008E1F06EB86071F26BE40B3438E1F06EB79
:10A5E000860602FA06F63343036311E010290FDAF8
:10A5F000C36AA1F10C0606EB86071F26BE40B343D3
:10A60000A1F10C0606EB860602FA06F63343C36296
:10A610000A2A0CDA046902EB42070726BE40B4435B
:10A6200002EB420605FA06F63443046111E0122AF1
:10A630000FDAC468A2F10A0606EB46070726BE40F9
:10A64000B443A2F10A0606EB460605FA06F63443C1
:10A65000C460F0BD0146C86C80B2704701F00102D1
:10A660001AB1826842F48002826001F002021AB1DB
:10A67000826842F4001282607047AAB101F48073CC
:10A680001BB1436843F48073436001F480631BB1E2
:10A69000436843F48063436001F00203CBB18368F5
:10A6A00043F00203836014E001F480731BB143683C
:10A6B00023F48073436001F480631BB1436823F487
:10A6C0008063436001F002031BB1836823F002033F
:10A6D0008360704710B501F073F901F067F910BDA0
:10A6E00010B504460548844207D140F2194001F0F4
:10A6F000B5FA40F2194001F0A1FA10BD0064004023
:10A70000014600208A69C2F30210704710B500218B
:10A71000837A012202FA03F13E4A126842F00102F2
:10A720003C4B1A603B4A1C3212688A43394B1C333B
:10A730001A60C289DAB9374A0C3212688A43354B3B
:10A740000C331A60C288344B03EA024243881A432E
:10A750004389304C403444F8332082882E4B03EA3E
:10A76000024203881A43438904EBC3035A60C28937
:10A77000012A1BD1274A0C3212680A43254B0C339D
:10A780001A600288244B03EA024243881A43438931
:10A79000204C403444F8332082881F4B03EA0242A5
:10A7A000C3881A43438904EBC3035A6082893AB9C8
:10A7B000184A121D12688A43164B1B1D1A6006E0C8
:10A7C000144A121D12680A43124B1B1D1A6002899B
:10A7D0003AB9104A143212688A430E4B14331A6085
:10A7E00006E00C4A143212680A430A4B14331A600A
:10A7F000027C012A06D1074A1C3212680A43054B23
:10A800001C331A60034A126822F00102014B1A60DD
:10A8100010BD0000006600400000FFFF70B502465A
:10A820004FF6FF730020146824F0020414601468CB
:10A8300044F00104146000E05B1E546804F001045D
:10A840000CB9002BF8D1546804F001040CB90020B5
:10A8500074E00C784FF0404505EA84744D784FF071
:10A86000407606EA05652C438D784FF4702606EA9B
:10A8700005452C43CD784FF4E00606EA05552C43F8
:10A880004D896D1EC5F309052C43D4610C79012C4B
:10A8900004D1146844F08004146003E0146824F0C8
:10A8A000800414604C79012C04D1146844F04004F5
:10A8B000146003E0146824F0400414608C79012CC7
:10A8C00004D1146844F02004146003E0146824F0F8
:10A8D00020041460CC79012C04D1146844F01004D5
:10A8E000146003E0146824F0100414600C7A012C46
:10A8F00004D1146844F00804146003E0146824F0E0
:10A90000080414604C7A012C04D1146844F0040447
:10A91000146003E0146824F004041460146824F044
:10A92000010414604FF6FF7300E05B1E546804F0EE
:10A9300001040CB1002BF8D103B1012070BD4269B4
:10A940008A434261704742690A434261704710B5C9
:10A9500000F5D87303EB01131B6803F004031372B3
:10A96000137A3BB900F5D87303EB01131B685B0D39
:10A97000136006E000F5D87303EB01131B68DB08D6
:10A98000536000F5D87303EB01131B6803F0020357
:10A99000537200F5DA7303EB01131B681B0AD374BF
:10A9A00000F5DA7303EB01131B6803F00F039372D6
:10A9B00000F5DC7303EB01131B68D37200F5DC7345
:10A9C00003EB01131B681C0A147300F5DC7303EB23
:10A9D00001131B681C0C547300F5DC7303EB0113AB
:10A9E0001B681C0E947300F5DE7303EB01131B68E8
:10A9F000D37300F5DE7303EB01131B681C0A147498
:10AA000000F5DE7303EB01131B681C0C547400F596
:10AA1000DE7303EB01131B681C0E947421B9C36829
:10AA200043F02003C36003E0036943F020030361A4
:10AA300010BD000030B502460B460021906800F0C2
:10AA40008060B0F1806F00D110E0906800F000608D
:10AA5000B0F1006F01D1012108E0906800F0805052
:10AA6000B0F1805F01D1022100E00321032901D16F
:10AA7000032030BD02F5C07000EB0110006800F04B
:10AA8000010402F5C07000EB01100460187A88B967
:10AA900018883B4C04EA40505C7A204302F5C074AD
:10AAA00004EB01142468204302F5C07404EB011484
:10AAB000206013E06FF00704586804EAC0001C7AB5
:10AAC00020435C7A204302F5C07404EB011424682F
:10AAD000204302F5C07404EB0114206002F5C2703B
:10AAE00000EB0110006820F00F0402F5C27000EBCB
:10AAF0000110046002F5C27000EB011000689C7A3E
:10AB0000204302F5C27404EB01142060987B4FF0DF
:10AB10007F4404EA00605C7B4FF47F0505EA04444F
:10AB200020431C7B2D1205EA04242043DC7A2043B9
:10AB300002F5C47404EB01142060987C2C0404EA30
:10AB400000605C7C2D0205EA044420431C7C2D122D
:10AB500005EA04242043DC7B204302F5C67404EBA1
:10AB60000114206002F5C07000EB0110006840F095
:10AB7000010402F5C07000EB01100460084678E79C
:10AB80000000E0FF10B5024632B1012A16D0022AB9
:10AB900020D0032A41D12EE000234B71CB718B7161
:10ABA00040F2FF334B8100230B724B7002238B70FA
:10ABB0000023CB700B714B720B7030E00123CB8103
:10ABC00000230B740B810B804B808B80CB808B819F
:10ABD0004B8124E0002005E0002401F10B031C540C
:10ABE000431CD8B20828F7D300238B724B600B723A
:10ABF0004B720B6013E0002005E0002401F10B0311
:10AC00001C54431CD8B20828F7D300238B724B6026
:10AC10000B72CB744B720B6001E000BFFEE700BF0C
:10AC200010BD00000349086000BF024909680029FF
:10AC3000FBD170479000002000EB400100BF0A1ECE
:10AC4000A1F10101FBD1704710B52C4B1B68834368
:10AC50002A4C2360231D1B688343241D2360231D6E
:10AC60001B688343241D2360231D1B688343241D0D
:10AC7000236011B101290ED105E0204B1B6803436D
:10AC80001E4C236008E01D4B1B1D1B6803431B4C1F
:10AC9000241D236000E000BF00BF22B1012A0FD0B5
:10ACA000022A27D119E0154B08331B680343134CC4
:10ACB00008342360231D1B688343241D23601AE08E
:10ACC0000E4B08331B6883430C4C08342360231D50
:10ACD0001B680343241D23600DE0084B08331B68E9
:10ACE0000343064C08342360231D1B680343241DC3
:10ACF000236000E000BF00BF10BD00000004014061
:10AD0000024909680143014A11607047000401408B
:10AD100001490860704700001404014001460748DB
:10AD2000006800EA010205481438006800EA0103DF
:10AD300012B10BB1012070470020FCE71404014060
:10AD400000B50346012200BF00F00CF802465B1E6E
:10AD5000012A01D1002BF7D1012A00D1042210468B
:10AD600000BD000000200A49C96801F0010109B1D5
:10AD700001200CE00649C96801F0100109B1032067
:10AD800005E00349C96801F0040101B102207047E0
:10AD90000020024000B50346012200BF00F00CF87D
:10ADA00002465B1E012A01D1002BF7D1012A00D1F6
:10ADB0000422104600BD000000200A49C96C01F0C1
:10ADC000010109B101200CE00649C96C01F0100134
:10ADD00009B1032005E00349C96C01F0040101B188
:10ADE0000220704700200240064A02EB90110968D9
:10ADF00000F01F0301229A401143024B03EB901213
:10AE0000116070470020024070B504460D460026D0
:10AE10002A480088B0F5007F35D22948844219D2EB
:10AE20004FF47020FFF78CFF0646002E43D12548D3
:10AE3000006940F001002349086125804FF470202B
:10AE4000FFF77EFF06461F48006920F001001D49FC
:10AE5000086130E04FF47020FFF79CFF064656BBB8
:10AE60001848006D40F001001649086525804FF430
:10AE70007020FFF78FFF06461248006D20F001009A
:10AE80001049086517E04FF47020FFF759FF064698
:10AE90008EB90C48006940F001000A49086125801C
:10AEA0004FF47020FFF74CFF06460648006920F07B
:10AEB000010004490861304670BD0000E0F7FF1F43
:10AEC000FFFF0708002002400848006940F08000AA
:10AED0000649086106480088B0F5007F04D9084695
:10AEE000006D40F0800008657047000000200240BF
:10AEF000E0F7FF1F30B5054636480088B0F5007F03
:10AF000048D9354885421ED24FF47020FFF718FF0C
:10AF10000446002C5BD13148006940F002002F4903
:10AF2000086108464561006940F0400008614FF43F
:10AF30007020FFF705FF04462848006920F0020052
:10AF40002649086143E04FF47020FFF723FF0446D1
:10AF5000002C3CD12148006D40F002001F490865DB
:10AF600008464565C06900F0020008B10846456121
:10AF70001A48006D40F04000184908654FF47020F1
:10AF8000FFF708FF04461548006D20F00200134942
:10AF900008651CE04FF47020FFF7D2FE0446B4B9F8
:10AFA0000E48006940F002000C49086108464561FE
:10AFB000006940F0400008614FF47020FFF7C0FEC8
:10AFC00004460648006920F0020004490861204652
:10AFD00030BD0000E0F7FF1FFFFF07080020024020
:10AFE0000C48006900F0800020B10B480949486016
:10AFF0000A4848600A480088B0F5007F09D905482A
:10B00000006D00F0800020B1034802494864034805
:10B01000486470470020024023016745AB89EFCDAB
:10B02000E0F7FF1F70B504460D4600262A48008849
:10B03000B0F5007F35D92948844219D24FF47020E9
:10B04000FFF77EFE0646002E43D12548006940F0FA
:10B0500001002349086125604FF47020FFF770FE5E
:10B0600006461F48006920F001001D49086130E0D4
:10B070004FF47020FFF78EFE064656BB1848006D51
:10B0800040F001001649086525604FF47020FFF775
:10B0900081FE06461248006D20F001001049086547
:10B0A00017E04FF47020FFF74BFE06468EB90C48B0
:10B0B000006940F001000A49086125604FF47020E2
:10B0C000FFF73EFE06460648006920F001000449ED
:10B0D0000861304670BD0000E0F7FF1FFFFF070862
:10B0E0000020024030B585B004460D461048007877
:10B0F000D8B114216846F7F73AF842F245100190AA
:10B1000004208DF8080000208DF8090001208DF83A
:10B110000A00E0B28DF80B0069460648FFF78AFC8A
:10B120004FF4FA70FFF788FD00BF204605B030BD30
:10B130000D0000200064004038B50020009000257C
:10B1400001220821254800F053F825480078401CCA
:10B15000C0B22349087000F001000870084600786A
:10B1600010B1012804D101E0002506E0012504E02A
:10B1700000201B490870002500BF00BF6946284613
:10B18000FFF7B5F9012800D021E00022082113487B
:10B1900000F02EF8BDF800004FF6FF7101EA001034
:10B1A00000907D2410E00F4830F81400BDF8001026
:10B1B000884207DBA4F1280040B20B49084A127804
:10B1C000885438BD601E84B2002CECD100BF002032
:10B1D0000549034A1278885400BFF2E70010014085
:10B1E00046000020E8C50008440000204161704787
:10B1F0000AB1016100E041617047000010B5002212
:10B200008B071C0F0F2303FA04F204290EDA204BDC
:10B210009B6893431E4CA36023469B688C07240FB6
:10B2200000FA04F423431A4CA3602FE008290EDA35
:10B23000174BDB689343164CE3602346DB688C07AF
:10B24000240F00FA04F42343114CE3601EE00C29A0
:10B250000EDA0F4B1B6993430D4C236123461B6988
:10B260008C07240F00FA04F42343094C23610DE0FA
:10B27000074B5B699343064C636123465B698C070C
:10B28000240F00FA04F42343014C636110BD000055
:10B2900000000140F0B5044616460025002201F0EA
:10B2A0000F0501F0100707B1354300201EE001270C
:10B2B00087401F40C7B122684FEA800C0F2707FA6A
:10B2C0000CF7BA43870005FA07F73A43282904D157
:10B2D000012787401F40676105E0482903D1012706
:10B2E00087401F4027612260471CB8B20828DED380
:10B2F000082022E0012787401F40E7B16268A0F1E3
:10B3000008074FEA870C0F2707FA0CF7BA43A0F19A
:10B310000807BF0005FA07F73A43282904D1012797
:10B3200087401F40676105E0482903D10127874016
:10B330001F4027616260471CB8B21028DAD3F0BD05
:10B3400002469068084008B1012070470020FCE7E1
:10B350000246D068084008B1012070470020FCE791
:10B36000F0B50A46002300240021002500F0004625
:10B37000B6F1004F02D11D4EF16901E01B4E71681C
:10B38000C0F3034583B200F44016B6F5401F08D160
:10B3900021F07061154E766826F07066134F7E605E
:10B3A00012E000F48016B6F5801F06D1032606FAD7
:10B3B00005F4A14341F0706106E0460D360103FA41
:10B3C00006F6B14341F0706122B1460D360103FA31
:10B3D00006F6314300F00046B6F1004F02D1034EAD
:10B3E000F16101E0014E7160F0BD0000000001401C
:10B3F00000F032FDFCF709FBFEF784F8FEF7B6F823
:10B40000F8F7AAFEFCF7CAFAFCF7F9FAF8F79AFC83
:10B41000F9F708FFF7F7E6FAFAF7E0F9F7F788FD2A
:10B42000F9F754FCFCF7B6FABB4800F061FA00BF2C
:10B43000F9F7ECF9F9F7A6F9FCF70AF9F9F71CFAAC
:10B44000FEF77CF8FEF7A8F8F9F77CFCF9F7A6FC04
:10B45000F9F7D4FAF9F7FEF9F8F780FCF9F720FCD0
:10B46000AE48007800F0400058B1AD48407801285F
:10B4700001D0FDF7D3FDA948006820F04000A7499E
:10B480000860A648007800F0800058B1A4484078D1
:10B49000022801D0FDF7CEFDA048006820F0800012
:10B4A0009E4908609D48008800F4807040B1FCF718
:10B4B000ADFC28B19948006820F480709749086075
:10B4C0009648008800F4007040B1FCF7A7FC28B152
:10B4D0009248006820F40070904908608F48008806
:10B4E00000F4806040B1FCF7A1FC28B18B480068F3
:10B4F00020F48060894908608848008800F4006072
:10B5000040B1FCF77BFC28B18448006820F400605F
:10B5100082490860FBF768F88048007800F0200056
:10B5200038B1FFF709FE7D48006820F020007B4914
:10B5300008607A48007800F0080038B1FCF77EFB1C
:10B540007648006820F00800744908607348007865
:10B5500000F0100038B1FCF7AFFB7048006820F035
:10B5600010006E4908606D48007800F0010038B1A5
:10B57000FBF7A8FD6948006820F0010067490860F2
:10B580006648007800F0040038B1FBF7FBFD634823
:10B59000006820F00400614908606048008800F4F9
:10B5A000805038B1FEF7EEF95C48006820F4805016
:10B5B0005A4908605948008800F4005038B1FEF735
:10B5C000E9F95648006820F400505449086053488F
:10B5D000008800F4804038B1FEF7E4F94F48006875
:10B5E00020F480404D4908604C48008800F4004039
:10B5F00038B1FEF7BFF94948006820F400404749D8
:10B6000008604648006800F4803038B1F7F7A4FAC3
:10B610004248006820F48030404908603F48006894
:10B6200000F4003038B1F7F7B7FA3C48006820F46E
:10B6300000303A4908603948006800F4802048B179
:10B64000F7F7EAF9F7F7CAFA3448006820F48020DF
:10B65000324908603148006800F4002038B1F7F73B
:10B66000E9F92E48006820F400202C4908602B4896
:10B67000006800F4001038B1F9F714FE274800689C
:10B6800020F40010254908602448006800F4801068
:10B6900028B12248006820F48010204908601F4823
:10B6A000006800F4800030B31C48006820F480007B
:10B6B0001A490860012080F3138800BF00BF00BF53
:10B6C00000BF00BF00BFBFF34F8F00BF00BF00BF70
:10B6D0001448006800F4E06013490843001D114954
:10B6E000086000BF00BF00BFBFF34F8F00BF00BFA7
:10B6F00000BF00BFFEE70948006800F40000002812
:10B700003FF496AE0548006820F400000349086045
:10B71000FDF760FB8CE6000044332211000000209E
:10B72000180100200CED00E00000FA052DE9F041C1
:10B7300003460D46164600240027A046244800680C
:10B7400000F4E060B0F5A06F15D006DCB0F5407FE6
:10B7500018D0B0F5806F19D110E0B0F5C06F06D0E9
:10B76000B0F5E06F12D100274FF0040815E0012773
:10B770004FF0030811E00227B8460EE003274FF010
:10B7800001080AE004274FF0000806E04FF4A0602B
:10B7900000F022F80227B84600BF00BFC7F104003E
:10B7A00005FA00F4C8F104010F20C84030400443FA
:10B7B00024010848C45403F01F0101208840591196
:10B7C000890001F1E021C1F80001BDE8F08100002D
:10B7D0000CED00E000E400E002490143024A116080
:10B7E000704700000000FA050CED00E00348006817
:10B7F00040F480700149086070470000007000400C
:10B800000E4A126822F003020C4B1A601A461268A4
:10B8100002431A600A4A126842F00402084B1A6096
:10B8200009B930BF02E040BF20BF20BF044A126800
:10B8300022F00402024B1A607047000000700040C2
:10B8400010ED00E010B540F20730FFF7CDFA10BD63
:10B850002DE9F041044620790004E17840EA012016
:10B86000A17840EA010707F100663046F6F78AFC46
:10B870000546FA2D00DDFA2520796071E078207107
:10B88000A078E0700020A0702A463146A01DF6F78F
:10B8900055FCA81DC0B2BDE8F08100004FF0FF309C
:10B8A00000F026F8012080F3138800BF00BF00BF1E
:10B8B00000BF00BF00BFBFF34F8F00BF00BF00BF7E
:10B8C0000948006800F4E06008490843001D064983
:10B8D000086000BF00BF00BFBFF34F8F00BF00BFB5
:10B8E00000BF00BFFEE700000CED00E00000FA051D
:10B8F0002DE9F04705461A48006800044FEA901900
:10B90000A9F5806000F10064D4F80880454501D1B4
:10B91000BDE8F08726686768FFF762FB08F1010061
:10B9200080B1FFF78FFF2046FFF7E4FAFFF78AFFA9
:10B9300031462046FFF776FBFFF784FF3946201D8E
:10B94000FFF770FB681C30B1FFF77CFF294604F15C
:10B950000800FFF767FBFFF7B7FA00BFD8E7000062
:10B96000E0F7FF1F0F4A51680F4A1140082814D210
:10B97000DFE800F004050607130A130B00BF00BF41
:10B9800000BF41EA803109E000BF20F004004FF021
:10B99000805242EA8032114300E000BF00BF014AFA
:10B9A0005160704700100240FF3FFFEF0348006AFC
:10B9B00020F4803001490862704700000010024006
:10B9C0000348006A40F48030014908627047000073
:10B9D000001002402DE9F04F8BB00746002009907F
:10B9E0003EA090E8004CC068CDE905BECDF810A09F
:10B9F00007900FF2EC0ADAE9000ACDE9020A0FF229
:10BA0000E00ADAE9000ACDE9000A38484068C0F3E4
:10BA100081000A900A9820B1012804D0022829D177
:10BA200003E0334928E0324926E03048406800F41A
:10BA30008038B8F5803F09D12D4C2C48406800F47F
:10BA40000039B9F5003F02D1641000E0294C2748C5
:10BA50004068C0F383422548406800F0006008B1A8
:10BA600042F010020F2A01D2921C00E0521C04FB8B
:10BA700002F101E01E4900BF00BF1C484068C0F34E
:10BA8000031504A8465D21FA06F318484068C0F380
:10BA9000022502A8465D23FA06FC14484068C0F35C
:10BAA000C2251DF8056023FA06F0089037B1012F72
:10BAB00006D0022F06D0032F0AD106E0099108E034
:10BAC000099306E0CDF824C003E00898099000E04F
:10BAD00000BF00BF09980BB0BDE8F08F0000000068
:10BAE00000000000010203040607080900100240DC
:10BAF00000127A0000093D000146074A02EB91104E
:10BB0000006801F01F0301229A40104008B1012093
:10BB100070470020FCE7000000100240064A02EBDC
:10BB20009011096800F01F0301229A401143024B53
:10BB300003EB90121160704700100240F0B506460A
:10BB4000002400270025182E51D003DC6EB3102EE0
:10BB50005DD106E0B6F5006F14D0B6F5106F56D182
:10BB600033E004E01120FFF7C7FF0546641C1DB950
:10BB70004FF6FF708442F5D11120FFF7BDFF00B1F1
:10BB8000012745E005E040F60100FFF7B5FF054657
:10BB9000641C1DB96FF07C408442F4D140F6010072
:10BBA000FFF7AAFF00B1012732E004E00120FFF710
:10BBB000A3FF0546641C15B9B4F5A06FF6D10120AA
:10BBC000FFF79AFF00B1012722E005E040F60110DF
:10BBD000FFF792FF0546641C15B90F488442F5D162
:10BBE00040F60110FFF788FF00B1012710E004E0E4
:10BBF0001920FFF781FF0546641C15B906488442E9
:10BC0000F6D11920FFF778FF00B1012700E000BF4F
:10BC100000BF3846F0BD0000FFFF0F00064A02EBF0
:10BC20009011096800F01F0301229A401143024B52
:10BC300003EB90121160704700100240064A02EBBD
:10BC40009011096800F01F0301229A409143024BB2
:10BC500003EB90121160704700100240064A02EB9D
:10BC60009011096800F01F0301229A401143024B12
:10BC700003EB90121160704700100240044A116AF1
:10BC800021F4407141EA0002014B1A627047000042
:10BC90000010024000B5024600F00CF8100C0449F8
:10BCA000086090B2091D086000F00EF800BD0000A9
:10BCB000202800400348006840F010000149086057
:10BCC00070470000042800400348006820F010007E
:10BCD00001490860704700000428004000B5024692
:10BCE000FFF7E8FF100C0449086090B2091D0860D6
:10BCF000FFF7EAFF00BD000018280040024909686C
:10BD00008143014A116070470428004001460448FD
:10BD10000068084008B1012070470020FCE70000DF
:10BD200004280040024909680143014A1160704734
:10BD30000028004000BF0348006800F020000028F1
:10BD4000F9D070470428004000B50246FFF7B2FF63
:10BD5000C2F303400349086090B2091D0860FFF771
:10BD6000B3FF00BD082800400648006820F0080026
:10BD70000449086000BF0348006800F0080000287C
:10BD8000F9D070470428004000200021264A12689C
:10BD900042F00102244B1A6000BF401C224A126884
:10BDA00002F0020111B9B0F5A06FF6D11E4A126877
:10BDB00002F002020AB900BFFEE71B4A52681A4BA2
:10BDC0005A601A4652685A601A46526842F48062B3
:10BDD0005A601A465268154B1A40134B5A601A465D
:10BDE0005268134B1A43104B5A601A46126842F0BD
:10BDF00080721A6000BF0C4A126802F00072002ABA
:10BE0000F9D0094A526822F00302074B5A601A46D9
:10BE1000526842F002025A6000BF034A526802F0C0
:10BE20000802002AF9D0704700100240FFFFC3F754
:10BE30000000280810B5FFF7A7FF10BD4FF0E02065
:10BE4000006920F002004FF0E02108610846006917
:10BE500020F001000861704710B5144800684FF4E5
:10BE60007A71B0FBF1F4601EB0F1807F01D3012044
:10BE70000FE0601E4FF0E02148610F214FF0FF30CE
:10BE8000FBF7C8FD00204FF0E02188610720086122
:10BE9000002008B100BFFEE70021481EFBF7BAFDF5
:10BEA0000020034908600349088010BDFC00002001
:10BEB0009000002098000020016841F0800101609E
:10BEC0007047000010B531B101293FD002297DD063
:10BED00003297CD1BFE0036A23F001030362836975
:10BEE00023F003038361036A148823430362036A14
:10BEF00023F002030362036A9488234303626A4BBC
:10BF0000984202D0694B98421FD1036A23F0040380
:10BF10000362036A548823430362036A23F008031D
:10BF20000362036AD48823430362436823F4807363
:10BF300043604368148923434360436823F40073D8
:10BF400043604368548923434360ABE0036A23F0B2
:10BF500010030362836923F440738361036A1488C6
:10BF600043EA04130362036A23F020030362036AB3
:10BF7000948843EA041303624B4B984202D04B4B24
:10BF8000984226D1036A23F040030362036A54886F
:10BF900043EA04130362036A23F080030362036A23
:10BFA000D48843EA04130362436823F48063436044
:10BFB0004368148943EA84034360436823F40063BD
:10BFC00043604368548943EA840301E002E068E087
:10BFD000436067E0036A23F480730362C36923F05C
:10BFE0000303C361036A148843EA04230362036AF8
:10BFF00023F400730362036A948843EA0423036210
:10C00000294B984202D0294B984223D1036A23F44A
:10C0100080630362036A548843EA04230362036A69
:10C0200023F400630362036AD48843EA04230362AF
:10C03000436823F4805343604368148943EA04133C
:10C040004360436823F4005343604368548943EAE0
:10C050000413436026E0036A23F480530362C36938
:10C0600023F44073C361036A148843EA0433036210
:10C07000036A23F400530362036A948843EA043397
:10C080000362094B984202D0084B984208D143689A
:10C0900023F4804343604368148943EA8413436074
:10C0A00000E000BF00BF10BD002C01400034014083
:10C0B00031B101290CD0022913D0032922D118E073
:10C0C000836923F0700383618369134383611AE0FA
:10C0D000836923F4E0438361836943EA0223836134
:10C0E00011E0C36923F07003C361C3691343C361E3
:10C0F00009E0C36923F4E043C361C36943EA02234F
:10C10000C36100E000BF00BF704731B1012906D014
:10C11000022906D0032908D105E0426306E08263C4
:10C1200004E0C26302E0026400E000BF00BF7047A9
:10C1300031B101290CD0022913D0032922D118E0F2
:10C14000836923F0080383618369134383611AE0E1
:10C15000836923F400638361836943EA0223836173
:10C1600011E0C36923F00803C361C3691343C361CA
:10C1700009E0C36923F40063C361C36943EA02238E
:10C18000C36100E000BF00BF704701460020486A5D
:10C19000704741627047000010B504463349601A89
:10C1A0008C4244D00CDCB4F1804F1CD03048204489
:10C1B00010B3B0F5806F28D0B0F5006F52D12DE0EC
:10C1C000B0F5806F3CD0B0F58E3F03D0B0F5923F14
:10C1D00048D13EE040F20B30FFF740FD40F20B301B
:10C1E000FFF72CFD3FE04FF48060FFF737FD4FF481
:10C1F0008060FFF723FD36E040F20140FFF72EFD9F
:10C2000040F20140FFF71AFD2DE040F20240FFF737
:10C2100025FD40F20240FFF711FD24E040F203400B
:10C22000FFF71CFD40F20340FFF708FD1BE040F262
:10C230000440FFF713FD40F20440FFF7FFFC12E05B
:10C2400040F20540FFF70AFD40F20540FFF7F6FC1B
:10C2500009E040F20D30FFF701FD40F20D30FFF72D
:10C26000EDFC00E000BF00BF10BD0000001000406A
:10C2700000FCFFBF016821F0010101607047016807
:10C2800041F00101016070470A888262294A9042A8
:10C2900020D0B0F1804F1DD0274A90421AD0274AB3
:10C2A000904217D0264A904214D0264A904211D08C
:10C2B000254A90420ED0254A90420BD0244A904203
:10C2C00008D0244A904205D0234A904202D0234A03
:10C2D00090420FD1026822F07002026002688B78EF
:10C2E00003F060031A43026002680B7903F0100345
:10C2F0001A4302608A68C262194A90420CD0194AF5
:10C30000904209D0026822F44072026002688B8970
:10C3100003F440731A430260064A904202D0094A6D
:10C32000904201D18A7B0263426942F0010242617C
:10C3300070470000002C014000040040000800404D
:10C34000000C004000340140004C0140005001400E
:10C350000054014000180040001C00400020004034
:10C360000010004000140040C2688A43C260704759
:10C37000C2680A43C260704702698A43026170471B
:10C380000246D06800EA01031069084010B10BB101
:10C39000012070470020FCE700210180418081805E
:10C3A0004FF6FF7181600021818181737047000029
:10C3B0002DE9F04704460D460027B846B946002649
:10C3C0001D49601A8C421CD006DC1C48204470B108
:10C3D000B0F5806F1FD10FE0B0F5806F16D0B0F5CB
:10C3E0006C4F18D10320FFF7F5FA074614E002203E
:10C3F000FFF7F0FA07460FE00220FFF7EBFA0746D7
:10C400000AE00220FFF7E6FA074605E00220FFF700
:10C41000E1FA074600E000BF00BF07EB5500B0FBA4
:10C42000F5F64FF6F07006EA000806F00F0948EA44
:10C430000900A060BDE8F087004C004000BCFFBFD1
:10C4400001464868C0F308007047C1F30802426023
:10C450007047000010B504462049601A8C4228D06D
:10C4600006DC1F48204490B1B0F5806F33D117E04F
:10C47000B0F5806F26D0B0F56C4F2CD140F20E3065
:10C48000FFF7ECFB40F20E30FFF7D8FB24E040F260
:10C490001140FFF7E3FB40F21140FFF7CFFB1BE039
:10C4A00040F21240FFF7DAFB40F21240FFF7C6FB02
:10C4B00012E040F21340FFF7D1FB40F21340FFF7C8
:10C4C000BDFB09E040F21440FFF7C8FB40F2144006
:10C4D000FFF7B4FB00E000BF00BF10BD004C004000
:10C4E00000BCFFBFC16841F40051C160704710B586
:10C4F000024602EB9110006801F01F040123A340E3
:10C50000184008B1012010BD0020FCE70A460021B8
:10C51000416921F400711143416170470A460021CD
:10C52000416921F4807111434161704710B5C1F335
:10C530008912825801F01F040123A3409A43C1F3DA
:10C540008913C25010BD10B5C1F38912825801F091
:10C550001F040123A3401A43C1F38913C25010BD25
:10C5600070B5024600230024C1F38910105801F071
:10C570001F060125B54000EA050302EB9150006853
:10C58000C1F304460125B54000EA050414B10BB11E
:10C59000012070BD0020FCE7C26822F4C062C260C6
:10C5A000C2680A43C26070470A460021C16821F090
:10C5B00004011143C1607047026922F440520261D4
:10C5C00002690A43026170470A460021C16821F0EE
:10C5D00008011143C1607047C26822F48052C260F2
:10C5E000C2680A43C260704720F682F5DCF42EF47C
:10C5F00078F3B9F2F1F120F145F061EF73EE7AEDE5
:10C6000077EC69EB51EA2DE9FEE7C4E67EE52CE420
:10C61000CFE266E1F0DF6FDEE2DC48DBA3D9F1D7E1
:10C6200034D66AD495D2B4D0C8CED1CCCFCAC1C882
:10C63000AAC688C45DC228C0E9BDA3BB54B9FDB673
:10C640009FB43AB2CFAF5EADE8AA6DA8EEA56BA3DA
:10C65000E5A05D9ED39B4799BB962E94A291178F20
:10C660008C8C048A7E87FB847C820080887D167B8C
:10C67000A8783F76DD7381712B6FDC6C946A536808
:10C680001A66E863BF619E5F855D745B6C596D5788
:10C6900076558953A451C84FF44D2A4C694AB04885
:10C6A00001475A45BC4327429A40163F9A3D273CD2
:10C6B000BC3A5939FE37AC3661351D34E232AD3102
:10C6C00080305B2F3C2E242D132C092B052A0829A2
:10C6D000112820273526502571249723C222F421C2
:10C6E0002A21652004C70008000000200401000082
:10C6F00098A0000808C80008040100200C320000BF
:10C70000A8A00008000000000000000000000000D9
:10C710000000010101000000000000000000000016
:10C7200000000100000000000000000000003100D7
:10C7300000000000000000030000000031000000C5
:10C7400000000000000000000000000000000000E9
:10C750000000000000000000000000000000FFFFDB
:10C76000FFFF0000000000000000000000000000CB
:10C7700000000000000000000000000000000000B9
:10C7800000000000000000000000000000000000A9
:10C790000000000000000000D2C6B75900000000F1
:10C7A000140E0100FC0F010014160100000000002F
:10C7B0000000000000000000000000000000000079
:10C7C0000000000000000000000000000000000069
:10C7D0000000000000000000000000000000000059
:10C7E0000000000000000000000000000000000049
:10C7F0000000000000000000000000000000000039
:08C8000000F36F0600000000C8
:0400000508002105C9
:00000001FF
